:10634000E5467006127AB58F4622E546B405061278
:106350003B6F8F4622E546B40B061270CF8F462264
:10636000E546B40A0612680D8F4622E546B40F06CC
:1063700012703B8F4622E546B414061261128F4616
:1063800022E546B419061279F88F4622E546B41E76
:1063900006127AC98F4622E546B42306126C188F7E
:1063A0004622E546B42806127B7E8F4622E546B497
:1063B0002D06127ADD8F4622E546B4320512732E81
:0363C0008F4622E3
:107AB500C20890061EE0FFA3E0901CECCFF0A3EFF8
:047AC500F07F052227
:103B6F00127B7A50477D047F011262B85008E53E00
:103B7F00B401037F0B227D047F021262B85008E567
:103B8F003EB402037F0B227D047F031262B85008FC
:103B9F00E53EB403037F0B227D047F041262B8500D
:103BAF0008E53EB404037F0B227F0A227F081275BB
:103BBF001550061253317F00227D057F051262B822
:103BCF005032901CEEE07002A3E070282046257D55
:103BDF00017F011262B84003023CE590066CE0FFE2
:103BEF007C0A7D70127273900610E0FFA3E0901CA8
:103BFF00EE023CAC7D067F051262B85031901CF08E
:103C0F00E07002A3E070272048247D017F0212623A
:103C1F00B84003023CE590066DE0FF7C0A7D9012F0
:103C2F007273900612E0FFA3E0901CF0806F7D0787
:103C3F007F051262B85031901CF2E07002A3E07061
:103C4F0027204C247D017F031262B84003023CE51C
:103C5F0090066EE0FF7C0A7DB0127273900614E03E
:103C6F00FFA3E0901CF280357D087F051262B850EB
:103C7F0033901CF4E07002A3E07029204F267D01E1
:103C8F007F041262B8504F90066FE0FF7C0A7DD020
:103C9F00127273900616E0FFA3E0901CF4CFF0A30E
:103CAF00EFF080327D077F061262B8500F30290C7B
:103CBF00901CECE07002A3E07002C22930380C9027
:103CCF001CECE07002A3E07002C238786CE6B40519
:093CDF00057F041260807F0522BC
:1070CF00203842900633E0901D10F0123346E53E13
:1070DF00B401062049247F0522E53EB40206204D67
:1070EF00197F0522E53EB4030620510E7F0522E5E8
:1070FF003EB404062054037F0522901D10E0D39464
:08710F000050C8D2387F0A22AB
:10680D00E53B700AE53EB40105753B018028E53B8B
:10681D00700AE53EB40205753B02801AE53B700A2D
:10682D00E53EB40305753B03800CE53B7008E53E82
:10683D00B40403753B047D077F061262B8500C7DCE
:10684D00077F061262B8501E30291B900650E0FFDC
:10685D007C067DF01272737D017F011262B85006C5
:09686D00120FB3122B647F0F22FD
:10703B00127B7A503F120FB3202F092030062031DC
:10704B0003303209E532700512770A800B786CE653
:10705B00B4050B7F03126080122B64120FB3202F29
:10706B001020300D20310A203207E5327003122B2D
:0A707B00647F0F2212770A7F1422AF
:10611200E4F53B900651E0FF7C077D101272737D1F
:10612200077F061262B8500C7D077F061262B850D4
:106132005E30295B786CE670047F018008786CE63B
:10614200B404077F021260808038786CE6B40704DA
:106152007601802E7D037F051262B85025901CF6D1
:10616200E07002A3E0701B900662E0FF7C097D30C4
:10617200127273900620E0FFA3E0901CF6CFF0A30A
:10618200EFF07F0612751550037F00227F19227DE2
:0E619200077F061262B850052029027F052201
:1079F8007D077F061262B850062029037F05229072
:0A7A08000630E0901D10F07F1E22F2
:107AC900901D10E070037F2322127B7A50037F0AF6
:047AD900227F1E22C8
:106C18007D047F071262B85041E53EB4010B90062F
:106C28005EE0FF7C087DB0802EE53EB4020B900646
:106C38005FE0FF7C087DD0801EE53EB4030B900624
:106C480060E0FF7C087DF0800EE53EB4040C900601
:106C580061E0FF7C097D10127273900631E0901D8F
:056C680010F07F28225E
:037B7E007F2D2236
:107ADD00901D10E070037F3222127B7A50037F0AD3
:047AED00227F2D22A5
:10732E003058037F32227D047F051262B8502890B8
:10733E001CF8E07002A3E0701E900663E0FF7C096B
:10734E007D50127273900622E0FFA3E0901CF8CFDE
:0C735E00F0A3EFF07F3222C2087F002273
:1073A300D224753D03123346122B64120FB3127BA2
:1073B3007A5009E53D600512334680F2E4F522F583
:1073C30023127B7A4009E53D600512334680F2E5DE
:0873D3003D70D2C224C2582211
:04000E0001000241AA
:0300030002693E51
:0B693E00C0E0C083C082C0D075D0084C
:10694900853082852F83E493FF204404C4540FFFCC
:10695900430FF08F80C284D28500C2870000D2879E
:10696900007580FF7580FEC284C28500C287000061
:106979000000D287007580FF30440CC2440530E521
:0B698900307006052F8002D244D2A817
:09699400D0D0D082D083D0E032D3
:03000B00021BB61F
:101BB600C0E0C0F0C083C082C0D075D008758CD894
:101BC600758A92D28C12421C12747AE531D3940033
:101BD60040051531021F40753111901D10E0D39458
:101BE600004003E014F0901D11E0D394004003E0A0
:101BF60014F0901D12E0D394004003E014F0901D01
:101C060013E0D394004003E014F0E532D39400408F
:101C16000215321541E541B40A004003021F3D900A
:101C26001C2CF8282873021F40021E91021E59021E
:101C36001E2C021DC2021D58021CEE021C84021C30
:101C460067021C4AD3901CEDE09400901CECE094D3
:101C5600005003021F40A3E024FFF0901CEC021F7B
:101C660031D3901CE9E09400901CE8E09400500306
:101C7600021F40A3E024FFF0901CE8021F317F0101
:101C86001277D24003021F40901CE1E09400901CA2
:101C9600E0E09400400CA3E024FFF0901CE0E03468
:101CA600FFF0D3901CEFE09400901CEEE09400400F
:101CB6000CA3E024FFF0901CEEE034FFF0D3901C60
:101CC600FBE09400901CFAE094005003021F407D54
:101CD600067F011262B84003021F40901CFBE024FD
:101CE600FFF0901CFA021F317F021277D2400302E6
:101CF6001F40901CE3E09400901CE2E09400400C2E
:101D0600A3E024FFF0901CE2E034FFF0D3901CF136
:101D1600E09400901CF0E09400400CA3E024FFF057
:101D2600901CF0E034FFF0D3901CFDE09400901C72
:101D3600FCE094005003021F407D067F021262B849
:101D46004003021F40901CFDE024FFF0901CFC02A3
:101D56001F317F031277D24003021F40901CE5E03B
:101D66009400901CE4E09400400CA3E024FFF09063
:101D76001CE4E034FFF0D3901CF3E09400901CF2D6
:101D8600E09400400CA3E024FFF0901CF2E034FF46
:101D9600F0D3901CFFE09400901CFEE094005003EA
:101DA600021F407D067F031262B84003021F409067
:101DB6001CFFE024FFF0901CFE021F317F04127707
:101DC600D24003021F40901CE7E09400901CE6E01E
:101DD6009400400CA3E024FFF0901CE6E034FFF0F2
:101DE600D3901CF5E09400901CF4E09400400CA302
:101DF600E024FFF0901CF4E034FFF0D3901D01E0E6
:101E06009400901D00E094005003021F407D067F61
:101E1600041262B84003021F40901D01E024FFF047
:101E2600901D00021F31D3901CEBE09400901CEA39
:101E3600E09400400CA3E024FFF0901CEAE034FF9D
:101E4600F0901D14E0D394005003021F40E014F0FC
:101E5600021F40D3901CF9E09400901CF8E0940017
:101E6600400CA3E024FFF0901CF8E034FFF0D39080
:101E76001CF7E09400901CF6E094005003021F400B
:101E8600A3E024FFF0901CF6021F31786CE6FF7089
:101E960003021F40EFB401059006188027786CE610
:101EA600FFB40219D3901CEBE09400901CEAE09476
:101EB60000403FA3E024FFF0901CEA806EEFB403DD
:101EC6001190061AE0FFA3E0901CEACFF0A3EFF012
:101ED6008020786CE6FFB4041ED3901CEBE09400DF
:101EE600901CEAE09400400AA3E024FFF0901CEA6C
:101EF6008039786C068043EF6405603E786CE6FFB7
:101F0600B4060D901CEA7402F0A37458F006802AF9
:101F1600EFB40726D3901CEBE09400901CEAE09403
:101F260000400EA3E024FFF0901CEAE034FFF080AE
:101F360009786C7600800375410A1279A54008126B
:101F460075D840031279C1D0D0D082D083D0F0D0DA
:021F5600E03277
:030013000261A0E7
:0D61A000C0E0C0F0C083C082C0D075D01038
:1061AD0075A0FFC284C285D287C286308018C2A472
:1061BD00C2A5D2A6C2A7E5A0540FF54AD2A7FF12D9
:1061CD00663DD286804F308118D2A4C2A5D2A6C218
:1061DD00A7E5A0540FF54AD2A7FF1263C3D286805C
:1061ED0034308218C2A4D2A5D2A6C2A7E5A0540FFE
:1061FD00F54AD2A7FF126443D2868019308316D296
:10620D00A4D2A5D2A6C2A7E5A0540FF54AD2A7FFE6
:05621D001264C3D286EB
:0B622200D0D0D082D083D0F0D0E0328A
:106BC100BF0113900632E0901D10F0901D10E0D32C
:106BD1009400404280F5BF0213900632E0901D11EF
:106BE100F0901D11E0D39400402C80F5BF03139069
:106BF1000632E0901D12F0901D12E0D39400401671
:106C010080F5BF0411900632E0901D13F0901D1322
:076C1100E0D3940050F722CC
:106C6D00304712205D0F900672E0FF7C0B7D3012D5
:106C7D007273D25D22304B12205F0F900673E0FFCE
:106C8D007C0B7D50127273D25F22304E1220600F3A
:106C9D00900674E0FF7C0B7D70127273D26022300F
:106CAD00521120610E900675E0FF7C0B7D901272E3
:046CBD0073D261220B
:1055B100303D1A204617900664E0FF7C097D701289
:1055C1007273D246C214C210C21CC21822304614D1
:1055D100203911900665E0FF7C097D90127273C23B
:1055E10046C23D22303E1A204817900666E0FF7CF5
:1055F100097DB0127273D248C215C211C21DC219FF
:1056010022304814203A11900667E0FF7C097DD0D2
:10561100127273C248C23E2230401A204C179006C3
:1056210068E0FF7C097DF0127273D24CC216C2127F
:10563100C21EC21A22304C14203B11900669E0FFB1
:105641007C0A7D10127273C24CC2402230421A2071
:105651004F1790066AE0FF7C0A7D30127273D24FB9
:10566100C217C213C21FC21B22304F13203C10901D
:10567100066BE0FF7C0A7D50127273C24FC2422258
:10517A00124102D28C7F0712751550051200168053
:10518A001212715F7F1F7E001277F990001FEFF0F5
:10519A001276327F08127515500512597A80FE90E0
:1051AA0006087402F0A37458F090060A7402F0A379
:1051BA007458F090060C7402F0A37458F090060E1E
:1051CA007402F0A37458F0900681E0FF7C0D7D1004
:1051DA00127273E4FFEFFD3395E0FC74302DF58213
:1051EA0074003CF583E0FE74F02DF582741A3CF5E8
:1051FA0083EEF00FBF08DED2081279C17545017F30
:10520A0001126080900618E0FFA3E0901CEACFF03C
:10521A00A3EFF0C2081279C1123346126340305923
:10522A0003124447305A03124334305B0312488A4C
:10523A00305E03124994124DA37D077F061262B8AD
:0C524A004002C2291255B1126C6D80CCDC
:104447007C007D80C2657F011236B550117F061250
:1044570075155002D2087F01121F580244E77C00ED
:104467007D70D2657F011236B55002800D7C007DCC
:1044770078D2657F011236B550077F011209418056
:104487005F7C007DA0D2657F011236B550117D0794
:104497007F061262B8500875450112773380417C58
:1044A700007DA8C2657F011236B550197D057F01D1
:1044B7001262B850107F061275155002D2087F019C
:1044C700124559801B7C007DB0C2657F011236B54D
:1044D700500E7F061275155002D2087F01124F93B6
:1044E700E4F54CAF4CEF3395E0FEEF7803C333CEE2
:1044F70033CED8F92400F58274013EAD82FCD26533
:104507007F011236B55038754501AF4CEF3395E052
:10451700FE74A02FF58274063EF583E0FFC007AF57
:104527004CEF3395E0FEEF7805C333CE33CED8F9A1
:1045370024F0F58274103EAD82FCD007126EB605EA
:104547004CC3E54C648094A84099C259C263126C6D
:01455700C1A2
:014558002240
:104334007F061275155002C2087D017F061262B80D
:10434400503D7C007D88C2657F021236B5500BD289
:10435400097F02121F58C20980257C007D70D26536
:104364007F021236B55002800D7C007D78D2657FC5
:10437400021236B55009D2097F02120941C20990CE
:10438400001FE030E1427C007DA0D2657F0212363E
:10439400B550147D077F061262B8500B12781F7552
:1043A4004502127733801E7C007DA8C2657F02120D
:1043B40036B550147D057F021262B8500B12781F77
:1043C4007F021245591279107D027F061262B8509D
:1043D4006AE4F54CAF4CEF3395E0FEEF7803C3335A
:1043E400CE33CED8F92400F58274013EAD82FCD2DE
:1043F400657F021236B55038754502AF4CEF3395E0
:10440400E0FE74A02FF58274063EF583E0FFC0073A
:10441400AF4CEF3395E0FEEF7805C333CE33CED8FF
:10442400F924F0F58274103EAD82FCD007126EB60A
:10443400054CC3E54C648094A84099C25AC26412E6
:024444006D15F4
:014446002253
:10488A007D037F061262B8503D7C007D90C2657F31
:10489A00031236B5500BD20E7F03121F58C20E8078
:1048AA00257C007D70D2657F031236B55002800DDB
:1048BA007C007D78D2657F031236B55009D20E7F0F
:1048CA0003120941C20E90001FE030E2427C007DD3
:1048DA00A0D2657F031236B550147D077F06126297
:1048EA00B8500B12781F754503127733801E7C006F
:1048FA007DA8C2657F031236B550147D057F031269
:10490A0062B8500B12781F7F031245591279107D35
:10491A00047F061262B8506AE4F54CAF4CEF339547
:10492A00E0FEEF7803C333CE33CED8F92400F58204
:10493A0074013EAD82FCD2657F031236B5503875DC
:10494A004503AF4CEF3395E0FE74A02FF582740651
:10495A003EF583E0FFC007AF4CEF3395E0FEEF78FA
:10496A0005C333CE33CED8F924F0F58274103EADA8
:10497A0082FCD007126EB6054CC3E54C648094A83D
:09498A004099C25BC228126D695C
:014993002201
:104994007D057F061262B8503D7C007D98C2657F1C
:1049A400041236B5500BD20C7F04121F58C20C806F
:1049B400257C007D70D2657F041236B55002800DCF
:1049C4007C007D78D2657F041236B55009D20C7F05
:1049D40004120941C20C90001FE030E3427C007DC8
:1049E400A0D2657F041236B550147D077F0612628B
:1049F400B8500B12781F754504127733801E7C0063
:104A04007DA8C2657F041236B550147D057F04125B
:104A140062B8500B12781F7F041245591279107D29
:104A2400067F061262B8506AE4F54CAF4CEF33953A
:104A3400E0FEEF7803C333CE33CED8F92400F582F9
:104A440074013EAD82FCD2657F041236B5503875D0
:104A54004504AF4CEF3395E0FE74A02FF582740645
:104A64003EF583E0FFC007AF4CEF3395E0FEEF78EF
:104A740005C333CE33CED8F924F0F58274103EAD9D
:104A840082FCD007126EB6054CC3E54C648094A832
:094A94004099C25EC22A126DBDF8
:014A9D0022F6
:106F5600BF010AC214C210C21CC2188025BF020A91
:106F6600C215C211C21DC2198018BF030AC216C2B9
:106F760012C21EC21A800BBF0408C217C213C21F58
:106F8600C21B90001FE0FF30E002D224EF30E10286
:0E6F9600D225EF30E202D226EF30E302D227FE
:016FA40022CA
:10663D008F4B7868E6C39450506E30496B7D077F61
:10664D00011262B8502B205C287868E6700D900618
:10665D003BE0B54B06203F03D23F22202F0D203FBC
:10666D000A7F01126F56753D02D22F900634E0F568
:10667D00327D087F061262B8501990063FE0B54B87
:10668D0006205C03D263220534E534AE33700E056B
:10669D0033800A0534E534AE337002053314F582C8
:0966AD008E83E54BF078680622AB
:1063C3008F4B7869E6C394505075304D727D077FCB
:1063D300021262B850327F021277D2502B205C280F
:1063E3007869E6700D90063BE0B54B06204103D279
:1063F300412220300D20410A7F02126F56753D0263
:10640300D230900634E0F5327D087F061262B85030
:106413001990063FE0B54B06205C03D26422053693
:10642300E536AE35700E0535800A0536E536AE35F0
:106433007002053514F5828E83E54BF078690622E8
:106443008F4B786AE6C3945050753051727D077F45
:10645300031262B850327F031277D2502B205C288C
:10646300786AE6700D90063BE0B54B06204303D2F5
:10647300432220310D20430A7F03126F56753D02DC
:10648300D231900634E0F5327D087F061262B850AF
:106493001990063FE0B54B06205C03D2282205384D
:1064A300E538AE37700E0537800A0538E538AE3764
:1064B3007002053714F5828E83E54BF0786A062265
:1064C3008F4B786BE6C3945050753054727D077FC1
:1064D300041262B850327F041277D2502B205C280A
:1064E300786BE6700D90063BE0B54B06204503D272
:1064F300452220320D20450A7F04126F56753D0256
:10650300D232900634E0F5327D087F061262B8502D
:106513001990063FE0B54B06205C03D22A22053AC8
:10652300E53AAE39700E0539800A053AE53AAE39D7
:106533007002053914F5828E83E54BF0786B0622E1
:10781F0090001FE0FF30E004D208D220EF30E104E7
:10782F00D209D221EF30E204D20ED222EF30E3049C
:05783F00D20CD223224F
:10791000C220C221C222C22390001FE0FF30E10238
:0F792000C209EF30E202C20EEF30E302C20C22C6
:106080008F4C30460302610D30480302610D204CF5
:106090007C204F79E54CB401197D017F051262B86F
:1060A000500C90065AE0FF7C087D30127273786CB9
:1060B0000622E54CB402177D027F051262B85048F3
:1060C00090065BE0FF7C087D50127273803AE54CCD
:1060D000B4041A7D027F051262B8500C90065DE090
:1060E000FF7C087D90127273786C760622E54C6412
:1060F00003701E7D027F051262B8500C90065CE0B2
:10610000FF7C087D70127273786C760122E4786CE3
:02611000F62275
:1079DD00EF1FAA0670011ED39400EA9400400BE439
:0A79ED00FDEDC394C850E90D80F7CA
:0179F700226D
:105A2F008F5D30695BE55DB40111D22090001FE0FE
:105A3F00F420E003305C44D2088040E55DB40211ED
:105A4F00D22190001FE0F420E103305C2ED20980B8
:105A5F002AE55DB40311D22290001FE0F420E20387
:105A6F00305C18D20E8014E55DB4040FD223900081
:105A7F001FE0F420E303305C02D20CAF5D026BC178
:105A8F00E55DB40110C22090001FE0F420E0033068
:105A9F005C41C20822E55DB40210C22190001FE0F4
:105AAF00F420E103305C2CC20922E55DB40310C27F
:105ABF002290001FE0F420E203305C17C20E22E5B3
:105ACF005DB4040FC22390001FE0F420E303305CA9
:045ADF0002C20C22D1
:105AE3008F5330675BE553B40111D22490001FE05C
:105AF300F420E003305C44D2088040E553B4021143
:105B0300D22590001FE0F420E103305C2ED20980FF
:105B13002AE553B40311D22690001FE0F420E203D8
:105B2300305C18D20E8014E553B4040FD2279000D2
:105B33001FE0F420E303305C02D20CAF53026BC1CD
:105B4300E553B40110C22490001FE0F420E00330B9
:105B53005C41C20822E553B40210C22590001FE045
:105B6300F420E103305C2CC20922E553B40310C2D4
:105B73002690001FE0F420E203305C17C20E22E5FA
:105B830053B4040FC22790001FE0F420E303305CFA
:045B930002C20C221C
:08290E008F538C548D558B563C
:10291600C265E55524FFF582E55434FFF583E0F5FD
:1029260058855582855483E0FFF559A3E0FEF55A94
:10293600EF14B40800505C90294B75F003A4C583CE
:1029460025F0C5837302296302296A0229710229C7
:102956007802297F02298602298D0229947557015A
:10296600D265802F755702D2658028755704D265C7
:102976008021755708D265801A755710D265801365
:10298600755720D265800C755740D26580057557FE
:1029960080D265EE24FE7003022A5B24F8605C2474
:1029A600096003022A6DE553B401059000208045B5
:1029B600E553B40205900021803BE553B40305902E
:1029C60000228031E553B404059000238027E553A7
:1029D600B40505900024801DE553B4060590002536
:1029E6008013E553B407059000268009E553640873
:1029F6007077900027E04557F0806EE553B40105E7
:102A06009000208045E553B40205900021803BE507
:102A160053B403059000228031E553B404059000B9
:102A2600238027E553B40505900024801DE553B4A3
:102A360006059000258013E553B40705900026800F
:102A460009E55364087022900027E0FFE557F4FE7D
:102A5600EF5EF08014E553B4080D855582855483E6
:102A6600E0FF125FECC265C265206503022B63E5D9
:102A760053B40109900020E0FD7F208060E553B447
:102A86000209900021E0FD7F218052E553B403093D
:102A9600900022E0FD7F228044E553B404099000B3
:102AA60023E0FD7F238036E553B40509900024E03A
:102AB600FD7F248028E553B40609900025E0FD7FBC
:102AC60025801AE553B40709900026E0FD7F26808D
:102AD6000CE553B4080C900027E0FD7F277E00121A
:102AE60072B3D2AFD269AF56125A2FAD58E4FF1265
:102AF60076B6AD59E4FF1276B6E55AB401047D38D0
:102B06008007E55AB40A077D367F061276B6E55386
:102B1600B408031276327D077F061262B8500B2086
:102B26002908C208C209C20EC20C7D017F011262C9
:102B3600B84002C2087D017F021262B84002C20993
:102B46007D017F031262B84002C20E7D017F04122E
:0D2B560062B84002C20CC269AF56125A2F7D
:012B6300224F
:045D85008F538D5457
:105D8900D269AF54125A2FAF54126BC1E553B40103
:105D9900059000208044E553B40205900021803A23
:105DA900E553B403059000228030E553B40405900F
:105DB90000238026E553B40505900024801CE55393
:105DC900B406059000258012E553B4070590002616
:105DD9008008E553B40806900027E0F555E55560BD
:105DE90025755701E4F556E55530E007AD57E4FF51
:105DF9001276B6E555C313F55505570556E556C34D
:105E0900940840E3800E7D187F021276B67D537F99
:0B5E1900021276B6C269AF54125A2F75
:015E2400225B
:021F58008F4DAB
:101F5A00E54D6401701E754E1B754F10900080E0B0
:101F6A00F550E54F2550F582E4354EF583E0F552FC
:101F7A0078688069E54D6402701E754E1B754F6066
:101F8A00900088E0F550E54F2550F582E4354EF58E
:101F9A0083E0F55278698045E54D6403701E754EFD
:101FAA001B754FB0900090E0F550E54F2550F58233
:101FBA00E4354EF583E0F552786A8021E54DB404A4
:101FCA001F754E1C754F00900098E0F550E54F259F
:101FDA0050F582E4354EF583E0F552786BE6F5511B
:101FEA00E55214B4090040030222F790200375F069
:101FFA0003A4C58325F0C5837302201E0220710243
:10200A0020C402211702216A0221BD0222100222E3
:10201A00610222B1E54F2550F582E4354EF583A3DE
:10202A00E0B40A18E5502402FFE433FEE551B5078F
:10203A000BE4B50607AD4D7F01022286AF507E0044
:10204A00EF2403FDEE33FCE5516D7001EC600302F1
:10205A0022F7EF254FFFEE354ECF2401FDE43FFC7A
:10206A00AB4D7F010222AEE54F2550F582E4354E95
:10207A00F583A3E0B40A18E5502402FFE433FEE531
:10208A0051B5070BE4B50607AD4D7F02022286AFB4
:10209A00507E00EF2403FDEE33FCE5516D7001EC38
:1020AA0060030222F7EF254FFFEE354ECF2401FDE4
:1020BA00E43FFCAB4D7F020222AEE54F2550F5828C
:1020CA00E4354EF583A3E0B40A18E5502402FFE490
:1020DA0033FEE551B5070BE4B50607AD4D7F0302A4
:1020EA002286AF507E00EF2403FDEE33FCE5516DEE
:1020FA007001EC60030222F7EF254FFFEE354ECF59
:10210A002401FDE43FFCAB4D7F030222AEE54F25DF
:10211A0050F582E4354EF583A3E0B40A18E550245D
:10212A0002FFE433FEE551B5070BE4B50607AD4DF2
:10213A007F04022286AF507E00EF2403FDEE33FCBB
:10214A00E5516D7001EC60030222F7EF254FFFEEB7
:10215A00354ECF2401FDE43FFCAB4D7F040222AE95
:10216A00E54F2550F582E4354EF583A3E0B40A180D
:10217A00E5502402FFE433FEE551B5070BE4B5064A
:10218A0007AD4D7F05022286AF507E00EF2403FD86
:10219A00EE33FCE5516D7001EC60030222F7EF2586
:1021AA004FFFEE354ECF2401FDE43FFCAB4D7F05DA
:1021BA000222AEE54F2550F582E4354EF583A3E0C1
:1021CA00B40A18E5502402FFE433FEE551B5070BC3
:1021DA00E4B50607AD4D7F06022286AF507E00EFBA
:1021EA002403FDEE33FCE5516D7001EC600302221D
:1021FA00F7EF254FFFEE354ECF2401FDE43FFCAB50
:10220A004D7F060222AEE54F2550F582E4354EF5A4
:10221A0083A3E0B40A17E5502402FFE433FEE55134
:10222A00B5070AE4B50606AD4D7F07804FAF507E6D
:10223A0000EF2403FDEE33FCE5516D7001EC600301
:10224A000222F7EF254FFFEE354ECF2401FDE43F82
:10225A00FCAB4D7F07804DE54F2550F582E4354EA6
:10226A00F583A3E0B40A18E5502402FFE433FEE53F
:10227A0051B5070BE4B50607AD4D7F08025D85AF82
:10228A00507E00EF2403FDEE33FCE5516D7001EC46
:10229A00705BEF254FFFEE354ECF2401FDE43FFC86
:1022AA00AB4D7F0802290EE54F2550F582E4354EE5
:1022BA00F583A3A3E07036E54F2550F582E4354E49
:1022CA00F583A3E024F96008147022AF4D0277ABBE
:1022DA00D2697F01125A2FAF4D126BC17D5E7F0208
:0D22EA001276B6C2697F01125A2F12597A7E
:0122F70022C4
:0436B5008C4D8D4E5D
:1036B900054EE54E7002054D14F5828C83E0F970D4
:1036C90003023857BF010875331B753410801FBFBB
:1036D900020875351B7536608014BF030875371BE2
:1036E9007538B08009BF040675391C753A00206524
:1036F900030237BDBF01087868E6696002C322BFCB
:1037090002087869E6696002C322BF0308786AE69D
:10371900696002C322BF0408786BE6696002C322AC
:10372900E4FEEEC39940030237BBEF6401701CE568
:103739004E2EF582E4354DF583E0FDE5342EF58214
:10374900E43533F583E06D6002C322EF6402701C37
:10375900E54E2EF582E4354DF583E0FDE5362EF58F
:1037690082E43535F583E06D6002C322EF640370AE
:103779001CE54E2EF582E4354DF583E0FDE5382E46
:10378900F582E43537F583E06D6002C322EF640406
:10379900701CE54E2EF582E4354DF583E0FDE53AE2
:1037A9002EF582E43539F583E06D6002C3220E02FD
:1037B900372BD322306503023858E4FEEEC3994013
:1037C90003023855EF6401701CE54E2EF582E4358D
:1037D9004DF583E0FDE5342EF582E43533F583E0DC
:1037E9006D6065C322EF6402701CE54E2EF582E41C
:1037F900354DF583E0FDE5362EF582E43535F58363
:10380900E06D6044C322EF6403701CE54E2EF5821F
:10381900E4354DF583E0FDE5382EF582E43537F5DD
:1038290083E06D6023C322EF6404701CE54E2EF51E
:1038390082E4354DF583E0FDE53A2EF582E435392C
:0F384900F583E06D6002C3220E0237C5D322C3A0
:01385800224D
:102B640090001FE0540FF55CB4010BE53EB4010383
:102B7400D21422C21422E55C6403702AE53EB40137
:102B840006D214D2108004C214C210E53EB402115D
:102B9400D2157D017F071262B84003022D7FD21146
:102BA40022C215C21122E55C6405702AE53EB40117
:102BB40006D214D21C8004C214C21CE53EB4031114
:102BC400D2167D027F071262B84003022D7FD21E07
:102BD40022C216C21E22E55C6409702AE53EB401D5
:102BE40006D214D2188004C214C218E53EB40411EB
:102BF400D2177D037F071262B84003022D7FD21BD8
:102C040022C217C21B22E55C6407704EE53EB40184
:102C140008D214D210D21C8006C214C210C21CE501
:102C24003EB40211D2157D017F071262B85002D260
:102C340011D21D8006C215C211C21DE53EB4031394
:102C4400D216D2127D027F071262B84003022D7F92
:102C5400D21E22C216C212C21E22E55C640B704E42
:102C6400E53EB40108D214D210D2188006C214C2B0
:102C740010C218E53EB40211D2157D017F0712621D
:102C8400B85002D211D2198006C215C211C219E578
:102C94003EB40413D217D2137D037F071262B840E7
:102CA40003022D7FD21B22C217C213C21B22E55C72
:102CB400640D704BE53EB40108D214D21CD21880C6
:102CC40006C214C21CC218E53EB40311D2167D021A
:102CD4007F071262B85002D21ED21A8006C216C2F0
:102CE4001EC21AE53EB40413D217D21F7D037F0718
:102CF4001262B84003022D7FD21B22C2178078E5EE
:102D04005C640F7076E53EB4010AD214D210D21C72
:102D1400D2188008C214C210C21CC218E53EB40204
:102D240013D2157D017F071262B85002D211D21D51
:102D3400D2198008C215C211C21DC219E53EB403DE
:102D440013D216D2127D027F071262B85002D21E2D
:102D5400D21A8008C216C212C21EC21AE53EB404B8
:102D640012D217D213D21F7D037F071262B8500B01
:0B2D7400D21B22C217C213C21FC21BD9
:012D7F002231
:100FB30090001FE0540FF55CB401167D017F011210
:100FC30062B8500A7F061275154003D20822C20880
:100FD30022E55C6403705BE53E640170257D017F5F
:100FE300011262B8500B7F061275154004D20880B7
:100FF30002C2087D017F021262B85003D20922C2E5
:101003000922E53E640260030214637D017F01123D
:1010130062B85004D2088002C2087D017F021262C6
:10102300B8500C7D017F071262B85003D20922C267
:101033000922E55C6405705BE53E640170257D0172
:101043007F011262B8500B7F061275154004D20857
:101053008002C2087D017F031262B85003D20E22C0
:10106300C20E22E53E640360030214637D017F0127
:101073001262B85004D2088002C2087D017F0312B5
:1010830062B8500C7D027F071262B85003D20E2261
:10109300C20E22E55C6409705BE53E640170257D48
:1010A300017F011262B8500B7F061275154004D2FE
:1010B300088002C2087D017F041262B85003D20C7B
:1010C30022C20C22E53E640460030214637D017FA7
:1010D300011262B85004D2088002C2087D017F0465
:1010E3001262B8500C7D037F071262B85003D20C12
:1010F30022C20C22E55C640760030211B5E53E647D
:101103000170347D017F011262B8500B7F061275A6
:10111300154004D2088002C2087D017F021262B822
:101123005004D2098002C2097D017F031262B850C4
:1011330003D20E22C20E22E53E640270367D017F89
:10114300011262B85004D2088002C2087D017F02F6
:101153001262B8500D7D017F071262B85004D209A4
:101163008002C2097D017F031262B85003D20E22AE
:10117300C20E22E53E640360030214637D017F0116
:101183001262B85004D2088002C2087D017F0212A5
:1011930062B85004D2098002C2097D017F03126242
:1011A300B8500C7D027F071262B85003D20E22C2E0
:1011B3000E22E55C640B6003021273E53E6401706A
:1011C300347D017F011262B8500B7F061275154002
:1011D30004D2088002C2087D017F021262B8500463
:1011E300D2098002C2097D017F041262B85003D282
:1011F3000C22C20C22E53E640270367D017F01128F
:1012030062B85004D2088002C2087D017F021262D4
:10121300B8500D7D017F071262B85004D2098002D5
:10122300C2097D017F041262B85003D20C22C20CA2
:1012330022E53E640460030214637D017F011262B0
:10124300B85004D2088002C2087D017F021262B83E
:101253005004D2098002C2097D017F041262B85092
:101263000C7D037F071262B85003D20C22C20C22FA
:10127300E55C640D6003021331E53E640170347D67
:10128300017F011262B8500B7F061275154004D21C
:10129300088002C2087D017F031262B85004D20E97
:1012A3008002C20E7D017F041262B85003D20C2269
:1012B300C20C22E53E640370367D017F011262B8E1
:1012C3005004D2088002C2087D017F031262B85025
:1012D3000D7D027F071262B85004D20E8002C20E47
:1012E3007D017F041262B85003D20C22C20C22E5A6
:1012F3003E640460030214637D017F011262B850EF
:1013030004D2088002C2087D017F031262B8500430
:10131300D20E8002C20E7D017F041262B8500C7D92
:10132300037F071262B85003D20C22C20C22E55C81
:10133300640F6003021463E53E640170437D017F23
:10134300011262B8500B7F061275154004D2088053
:1013530002C2087D017F021262B85004D2098002E2
:10136300C2097D017F031262B85004D20E8002C20B
:101373000E7D017F041262B85003D20C22C20C22EC
:10138300E53E640270457D017F011262B85004D2CC
:10139300088002C2087D017F021262B8500D7D01F0
:1013A3007F071262B85004D2098002C2097D017F0F
:1013B300031262B85004D20E8002C20E7D017F0474
:1013C3001262B85003D20C22C20C22E53E640370B1
:1013D300457D017F011262B85004D2088002C20821
:1013E3007D017F021262B85004D2098002C2097DD6
:1013F300017F031262B8500D7D027F071262B8505D
:1014030004D20E8002C20E7D017F041262B8500323
:10141300D20C22C20C22E53E640470447D017F019C
:101423001262B85004D2088002C2087D017F021202
:1014330062B85004D2098002C2097D017F0312629F
:10144300B85004D20E8002C20E7D017F041262B82E
:10145300500C7D037F071262B85003D20C22C20CDA
:011463002266
:1078AF007F011277D25010C209C20EC20C7F06128E
:1078BF007515500CC208227F011277D24002C20800
:0178CF002296
:107A2C007F021277D25007C209C20EC20C227F020B
:087A3C001277D24002C20922B8
:107A44007F031277D25007C209C20EC20C227F03F1
:087A54001277D24002C20E229B
:107A5C007F041277D25007C209C20EC20C227F04D7
:087A6C001277D24002C20C2285
:10699D000500050105030507050F051F051E051C4F
:1069AD00051805100201040E040A03060101040B6B
:1069BD000304040F020304010302040D020002028A
:1069CD00030004090404030503070100030304077E
:1069DD00030104060402040C051605150000061536
:0E69ED00062A060C06380633061E061206178A
:10525600203737900640E004F519D36480948150D6
:1052660003025330D3E5196480948F400375190FF8
:1052760090063DE0FF123E5C90063EE0F518E4F530
:105286001ED237C262C257C24A22304A6030621604
:10529600152EE52ED394004003025330C2CAC262D3
:1052A600D25785182E2230570E152EE52ED3940090
:1052B6005078C262C25722AF1C151CEF700BC24A4F
:1052C600E51825E0F52ED25722E51D30E0058518B4
:1052D6002E8008E51875F003A4F52EAF1D7801EFB2
:1052E60008800103D8FDF51DD262D2CA22D519085D
:1052F600C237E4F53DC25822051E7440251EF582CC
:10530600E43406F583E025E0249DF582E43469F56E
:1053160083E493540FF51C740193F51D700AD2575C
:0A532600E51825E025E0F52ED24A37
:01533000225A
:105EBE0020371A90063DE0FF123E5C90063EE0F55C
:105ECE001AE4F51ED237C262C257C24A22304A596C
:105EDE00306213152EE52ED39400506BC2CAC262E7
:105EEE00D257851A2E2230570E152EE52ED394003A
:105EFE005055C262C25722AF1C151CEF7007C24A22
:105F0E00C237F53D22E51D30E005851A2E8008E5E5
:105F1E001A75F003A4F52EAF1D7801EF088001036A
:105F2E00D8FDF51DD262D2CA22E53F25E0249DF5AB
:105F3E0082E43469F583E493FA740193FBEA540F17
:075F4E00F51CEBF51DD24A22
:015F55002229
:107AF100C3EF648094A15008EF25E025E0F52E2224
:047B0100E4F52E2257
:10744600BF010790063E7418F022BF020790063E61
:107456007412F022BF030590063E8014BF04079005
:10746600063E740BF02290063EBF05047409F02216
:04747600740CF02280
:103E5C00EF14B420004003023FAF903E7475F003A2
:103E6C00A4C58325F0C58373023ED4023EDB023E1B
:103E7C00E2023EE9023EF0023EF7023EFE023F0540
:103E8C00023F0C023F13023F1A023F21023F28025D
:103E9C003F2F023F36023F3D023F44023F4B023F61
:103EAC0052023F59023F60023F67023F6E023F756C
:103EBC00023F7C023F83023F8A023F91023F930202
:103ECC003F9A023FA1023FA875CB8E75CAC62275D8
:103EDC00CB9575CA772275CB9B75CA692275CBA019
:103EEC0075CABA2275CBA675CA332275CBAB75CA07
:103EFC00632275CBB075CA022275CBB475CAA322E6
:103F0C0075CBB875CAFA2275CBBC75CAD82275CBDD
:103F1C00C075CAA82275CBC475CA362275CBC775B5
:103F2C00CA862275CBCA75CABC2275CBCD75CAB4EC
:103F3C002275CBD075CA762275CBD375CA30227553
:103F4C00CBD575CAB22275CBD875CA132275CBDA0C
:103F5C0075CA522275CBDC75CA7D2275CBDD75CA4C
:103F6C006E2275CBE075CA542275CBE275CA1B2242
:103F7C0075CBE375CAC32275CBE575CA5E2275CBCA
:103F8C00E675CADA22801C75CBE875CA902275CB0F
:103F9C00EA75CAD92275CBEC75CA092275CBED75B9
:0A3FAC00CA292275CBE875CA41222C
:1071A700EFC39400403FEF9408503AE4FEEF75F0C8
:1071B70008A42430F582E43400F583E5822EF582B5
:1071C700E43583F583E0FCED75F008A424E8F58247
:1071D700E4341AF583E5822EF582E43583F583ECF2
:0571E700F00EBE08C817
:0171EC002280
:105FEC008F5BE55B6405701D200A0DD20A7FF47E81
:105FFC00011279DDC20A8074C20A7FF47E01127923
:10600C00DDD20A8067E55B6406701D200B0DD20B98
:10601C007FF47E011279DDC20B800BC20B7FF47E04
:10602C00011279DDD20B8044E55B6407701D200FF3
:10603C000DD20F7FF47E011279DDC20F800BC20FDF
:10604C007FF47E011279DDD20F8021E55B6408704C
:10605C0022200D0DD20D7FF47E011279DDC20D8050
:10606C000BC20D7FF47E011279DDD20D7FF47E011F
:04607C001279DD2296
:104DA300A233B330B401B350357D017F081262B82A
:104DB3005027A233B35010A2B4B3500B900652E065
:104DC300FF7C077D30800F30330F30B40C900653D7
:104DD300E0FF7C077D50127273A2B4B39233A23406
:104DE300B330B501B350357D027F081262B8502746
:104DF300A234B35010A2B5B3500B900654E0FF7C1D
:104E0300077D70800F30340F30B50C900655E0FFEE
:104E13007C077D90127273A2B5B39234A235B3307E
:104E2300B701B350357D037F081262B85027A2350E
:104E3300B35010A2B7B3500B900656E0FF7C077D2A
:104E4300B0800F30350F30B70C900657E0FF7C076A
:104E53007DD0127273A2B7B39235A236B330B601C6
:104E6300B350357D047F081262B85027A236B35081
:104E730010A2B6B3500B900658E0FF7C077DF0807C
:104E83000F30360F30B60C900659E0FF7C087D10CA
:094E9300127273A2B6B39236222A
:10763200900027E0FF30E404D20A8002C20AEF3051
:10764200E504D20B8002C20BEF30E604D20F8002B7
:0B765200C20FEF30E703D20D22C20D83
:01765D00220A
:1073DB0090063CE0FF602E20370F6029123E5CD2F6
:1073EB00CAD237D262752E1422E52ED394004003F5
:1073FB00152E22206208D2CA752E14D26222C2CA5E
:06740B00752E7DC2622215
:107411002037127F1C123E5CD2CAD237D262752E3F
:1074210064751B3C22E52ED394004003152E22AF38
:107431001B151BD3EF648094804004752E6422C217
:0474410037E4F53DFA
:017445002224
:104E9C0020371C754006E53E75F008A424E8F58221
:104EAC00E4341AF583E06003D23722E4F53D22E5C1
:104EBC002ED394004003152E22C2CA1540E540148F
:104ECC007003024F5714606F14604014602E14600E
:104EDC0003024F8BE53E75F008A424E8F582E43418
:104EEC001AF583E0FF7003F53D22123E5CE53E753A
:104EFC00F008A424E9F582E4341A8079E53E75F0D3
:104F0C0008A424EAF582E4341A80397408441B702E
:104F1C0003F53D22E53E75F008A424EBF582E4345C
:104F2C001AF583E0FF123E5CE53E75F008A424EC14
:104F3C00F582E4341A803EE53E75F008A424EDF5C4
:104F4C0082E4341AF583E0FF027AF17420441B707A
:104F5C0003F53D22E53E75F008A424EEF582E43419
:104F6C001AF583E0FF123E5CE53E75F008A424EFD1
:104F7C00F582E4341AF583E0FF127AF1D2CA22E406
:074F8C00F53DC2CAC2372245
:10747A00E53D14601C14601C14601C14601F146029
:10748A001F2405701EC2CAC237C262C257E4F54041
:10749A0022024E9C0273DB125256D25822027411F7
:0474AA00125EBE228E
:1075D800E52365437004E5226542601F85224285E4
:1075E8002343C2A4D2A5C2A6C2A700AF23127A8A97
:0D75F800E522FF127A8A00D2A7D322C32217
:1079A500E52465446014852444D2A4D2A5C2A6C2A8
:0C79B500A7AF24127A8AD2A7D322C322E3
:1079C100E521653C601485213CD2A4C2A5C2A6C2B2
:0C79D100A7AF21127A8AD2A7D322C322CA
:10410200E4F54CF54D754E1E754FFF854D82854C7D
:1041120083E0F5506350FFE550F0E0655060031214
:104122007B816350FF854D82854C83E550F0E065CD
:10413200506003127B81054DE54D7002054CE54F41
:10414200154F7002154ED3E54F9400E54E94005082
:10415200BAE4F54CF54DF54EF54FE54D254FF58298
:10416200E54C354EF583E4F0054FE54F7002054E00
:10417200B4FFE7E54EB41EE275985A758921758839
:1041820045758845758DE775878075C90275331B3E
:1041920075341075351B75366075371B7538B075FB
:1041A200391C753A0075B701D2A9D2A8D2AA9006D5
:1041B20000E0FFA3E0901CE0CFF0A3EFF090060236
:1041C200E0FFA3E0901CE2CFF0A3EFF0900604E042
:1041D200FFA3E0901CE4CFF0A3EFF0900606E0FF0F
:1041E200A3E0901CE6CFF0A3EFF0901CFA7417F056
:1041F200A37499F0901CFC7417F0A37499F0901CAE
:10420200FE7417F0A37499F0901D007417F0A37454
:0942120099F0D291D2AF1276E0CE
:01421B002280
:027B810080FE84
:10751500C2AFC284D285BF060AC286E580A2E192C7
:10752500698018BF070AC286E580A2E29269800BCE
:10753500BF0808C286E580A2E39269D286D2AFA2CF
:0175450069DC
:017546002222
:1062B800BF0107900020E0FE8048BF020790002140
:1062C800E0FE803EBF0307900022E0FE8034BF045A
:1062D80007900023E0FE802ABF0507900024E0FE17
:1062E8008020BF0607900025E0FE8016BF070790B4
:1062F8000026E0FE800CBF0807900027E0FE800221
:10630800E4FEBD0103EE1322BD0204EEA2E122BDAC
:106318000304EEA2E222BD0404EEA2E322BD0504BA
:10632800EEA2E422BD0604EEA2E522BD0704EEA219
:07633800E622BD0802EE336E
:01633F00223B
:024F93008F4D40
:104F95009000B0E0F54EE54D64017037E54E240212
:104FA500FFE433FE7868E66F7001EE600302508817
:104FB5007410254EF582E4341BAF82F5508F51D223
:104FC500697F01125A2F12796B123859C2697F0114
:104FD500025085E54D64027037E54E2402FFE43347
:104FE500FE7869E66F7001EE6003025088746025F3
:104FF5004EF582E4341BAF82F5508F51D2697F02A2
:10500500125A2F12796B123859C2697F02025085E4
:10501500E54D64037033E54E2402FFE433FE786A00
:10502500E66F7001EE705C74B0254EF582E4341BBA
:10503500AF82F5508F51D2697F03125A2F12796BC7
:10504500123859C2697F038037E54D64047034E531
:105055004E2402FFE433FE786BE66F7001EE702399
:105065007400254EF582E4341CAF82F5508F51D281
:10507500697F04125A2F12796B123859C2697F045D
:03508500125A2F8D
:015088002205
:043859008F4FE4FDAC
:02385D008D5785
:10385F0075F020EFA42460F582E5F03403AF82F514
:10386F005A8F5BF583E0F558D3940050030239E586
:10387F00E558941040030239E5E557704C7FF47E0C
:10388F00011279DDE55825E0F558755901E5582401
:10389F0001FFE433FEC3E5599FEE6480F87480980E
:1038AF0040030239E5E55B2559F582E4355AF58386
:1038BF00E0FFE55B2559F582E4355AF583A3E0FD7A
:1038CF001276B60559055980C4E5576401707AC25E
:1038DF002B7FF47E011279DDE55825E0F5587559F7
:1038EF0001E5582401FFE433FEC3E5599FEE6480E0
:1038FF00F874809840030239E5E55B2559F582E4B9
:10390F00355AF583E0FFE55B2559F582E4355AF525
:10391F0083A3E0FD1276B690001FE0FF30E0063083
:10392F004903C22022EF30E106304D03C22122EFBE
:10393F0030E206305103C22222EF30E30630540347
:10394F00C22322055905598098E557640260030286
:10395F0039E5C22BC22CC22DC22E7FF47E01127903
:10396F00DDE55825E0F558755901E5582401FFE4C8
:10397F0033FEC3E5599FEE6480F87480985057E585
:10398F005B2559F582E4355AF583E0FFE55B255950
:10399F00F582E4355AF583A3E0FD1276B690001F49
:1039AF00E030E005303902802290001FE030E10561
:1039BF00303A02801690001FE030E205303B028063
:1039CF000A90001FE030E308303C05C2200273A3C9
:0639DF0005590559809412
:0139E50022BF
:024559008F4D84
:10455B00C2659000A8E0FFE54DB401167868E6FE51
:10456B00D39F400EEE9FF55074102FF582E4341B51
:10457B00804FE54DB402167869E6FED39F400EEEF0
:10458B009FF55074602FF582E4341B8034E54DB4F5
:10459B000316786AE6FED39F400EEE9FF55074B07B
:1045AB002FF582E4341B8019E54DB4041C786BE6BF
:1045BB00FED39F4014EE9FF55074002FF582E43428
:1045CB001CAF82F5518F52D265206503024669D22A
:1045DB0069AF4D125A2F7FF47E011279DD7D207F5A
:1045EB00051276B67D1A7F081276B67FC87E00124A
:1045FB0079DDE4F54EE54EC39550505B0552E5521F
:10460B00AE517002055114F5828E83E0F54F603682
:10461B0024F5601414601714601A14601D146020C4
:10462B0024057028E4FD80277D5F7F0780227D5E57
:10463B007F06801C7D0A7F0280167D327F028010F0
:10464B007D467F02800A7D0A7F038004AD4FE4FF25
:0E465B001276B6054E809EC269AF4D125A2FE0
:01466900222E
:1077330030290F900671E0FF7C0B7D10127273B23B
:107743002922202912900670E0FF7C0A7DF0127234
:0877530073B229E4786CF62200
:105F56007D3F7F091276B67D507F081276B6900097
:105F66000EE493FDE4FF1276B67D5B7F061276B6ED
:105F760090000FE493FDE4FF1276B6900010E493D0
:105F8600FDE4FF1276B6900011E49324BFB4080036
:105F96005053905FA675F003A4C58325F0C583739F
:105FA600025FBE025FC2025FC6025FCC025FD20220
:105FB6005FD8025FDE025FE47D0A80067D328002E2
:105FC6007D467F02801C7D0A7F0380167D287F0325
:105FD60080107D467F03800A7D0A7F0480047D2829
:065FE6007F041276B622D2
:1077AB008F53D269125A2F7D4B7F021276B67D040E
:1077BB00E4FF1276B67D387F041276B6125F56C29E
:0777CB0069AF53125A2F228F
:0B796B00855182855083E0FFA3E0FD02
:10797600BF0A02E4FFBD0A02E4FDEF75F00AA42D7A
:02798600FF22DE
:10533100C265D208D2207FF47E011279DD7D2E7FF5
:10534100031276B67D607F021276B6C208C22012C1
:1053510033467F0812751540030253FD3049F012A0
:1053610033462049FA7868E6640770427E007F7010
:1053710075331B7534108F828E837407F07D01E5C0
:10538100342DF582E43533F583E58224FFF582E59A
:105391008334FFF583E0F9EF2DF582E43EF583E9EF
:1053A100F00DBD08DAD2657F647E001279DD7F08D9
:1053B1001275155047206503025333D208D2207F5E
:1053C100F47E011279DD7D607F021276B67D327F37
:1053D100061276B67D1E7F051276B6C208C2207C03
:1053E100007D707B087F787E001267A07F081275B0
:1053F1001550097F327E001279DD80F0126CC17F79
:06540100647E001279DD5B
:015407002282
:10770A00E4F53DC258C258F532302F05C22FC23FA8
:10771A0022303005C230C24122303105C231C24363
:09772A0022303204C232C24522B1
:10421C007580FFC286E580540FFFC285E580C454CB
:10422C00F04FF520D2867D027F011262B840107DDE
:10423C00037F011262B84007300004D23980287D18
:10424C00027F011262B8500A300007300104D239E3
:10425C0080157D037F011262B8500A2000033001E3
:10426C0004D2398002C2397D027F021262B840103A
:10427C007D037F021262B84007300204D23A8028D4
:10428C007D027F021262B8500A300207300304D25A
:10429C003A80157D037F021262B8500A2002033067
:1042AC000304D23A8002C23A7D027F031262B84004
:1042BC00107D037F031262B84007300404D23B80A8
:1042CC00287D027F031262B8500A300407300504BF
:1042DC00D23B80157D037F031262B8500A20040381
:1042EC00300504D23B8002C23B7D027F041262B8CF
:1042FC00400F7D037F041262B84006300603D23CA7
:10430C00227D027F041262B8500930060630070382
:10431C00D23C227D037F041262B850092006033080
:07432C000703D23C22C23C52
:014333002267
:10334600202B6A20391C205019901CFAE07002A329
:10335600E0700B7D067F011262B85002D247C24967
:10336600804B30392130501E901CE0E07002A3E003
:10337600700B7D087F011262B85002D23D306302A5
:10338600D259D2498027303908205005126CC180A5
:103396001C203919305016C249C250C214C210C27C
:1033A6001CC2181278AF7868E66002D259202C71D8
:1033B600203A1C205319901CFCE07002A3E0700B0D
:1033C6007D067F021262B85002D24BC24D80523047
:1033D6003A28305325901CE2E07002A3E070127D7B
:1033E600087F021262B850097F021277D25002D2C9
:1033F6003E306402D259D24D8027303A0820530518
:10340600126D15801C203A19305316C24DC253C294
:1034160015C211C21DC219127A2C7869E66002D251
:103426005A202D71203B1C205519901CFEE070027D
:10343600A3E0700B7D067F031262B85002D24EC223
:10344600518052303B28305525901CE4E07002A391
:10345600E070127D087F031262B850097F0312776D
:10346600D25002D240302802D259D2518027303B66
:1034760008205505126D69801C203B19305516C26F
:1034860051C255C216C212C21EC21A127A44786AB4
:10349600E66002D25B202E6D203C1B205618901D44
:1034A60000E07002A3E0700B7D067F041262B85044
:1034B60002D252C25422303C27305624901CE6E0F9
:1034C6007002A3E070127D087F041262B850097F73
:1034D600041277D25002D242302A02D259D2542252
:1034E600303C06205603026DBD203C19305616C2EC
:1034F60054C256C217C213C21FC21B127A5C786B23
:06350600E66002D25E2225
:047B7A0012508922FA
:1050890090001FE0540FFFBF010B304906203D037C
:10509900025150C322EF64037014304906203D03C6
:1050A900025150304D06203E0302515BC322EF648A
:1050B900057014304906203D030251503051062035
:1050C9004003025166C322EF640970133049052079
:1050D9003D028073305406204203025171C322EF0E
:1050E9006407701A304905203D02805B304D052068
:1050F9003E02805E3051052040028061C322EF6488
:105109000B701A304905203D02803C304D05203E88
:1051190002803F305405204202804DC322EF640DC6
:10512900701A304905203D02801D3051052040028A
:10513900802B305405204202802EC322EF640F7069
:105149002E304908203D05753E01D322304D0820F7
:105159003E05753E02D322305108204005753E03B5
:10516900D322305408204205753E04D322C322C3FA
:015179002213
:1077D200BF010690001FE01322BF020790001FE0C6
:1077E200A2E122BF030790001FE0A2E222BF04062B
:0777F20090001FE0A2E3225A
:106CC1007868E6602275331B753410E4FFE5342FD4
:106CD100F582E43533F583E4F00FBF50F075331BD3
:106CE100753410E47868F6900600E0FFA3E0901C8C
:106CF100E0CFF0A3EFF0900608E0FFA3E0901CFACC
:106D0100CFF0A3EFF0C246C247C25DC23DC263C22B
:036D11003FD2501E
:016D1400225C
:106D15007869E6602275351B753660E4FFE5362F28
:106D2500F582E43535F583E4F00FBF50F075351B7A
:106D3500753660E47869F6900602E0FFA3E0901CE2
:106D4500E2CFF0A3EFF090060AE0FFA3E0901CFC71
:106D5500CFF0A3EFF0C248C24BC25FC23EC264C2CD
:036D650041D253C5
:016D68002208
:106D6900786AE6602275371B7538B0E4FFE5382F7D
:106D7900F582E43537F583E4F00FBF50F075371B22
:106D89007538B0E4786AF6900604E0FFA3E0901C39
:106D9900E4CFF0A3EFF090060CE0FFA3E0901CFE17
:106DA900CFF0A3EFF0C24CC24EC260C240C228C2AB
:036DB90043D2556D
:016DBC0022B4
:106DBD00786BE6602275391C753A00E4FFE53A2FD1
:106DCD00F582E43539F583E4F00FBF50F075391CC9
:106DDD00753A00E4786BF6900606E0FFA3E0901C90
:106DED00E6CFF0A3EFF090060EE0FFA3E0901D00BC
:106DFD00CFF0A3EFF0C24FC252C261C242C22AC24B
:036E0D0045D25615
:016E1000225F
:10597A00C208C209C20EC20C1279C1C265D25CE465
:10598A00F53D7FE87E031279DDC298C2AF75567F76
:10599A00755596755498755300785374FF12595C6F
:1059AA00E4FBFAF9F8C3125949504430983E120000
:1059BA0006127B3CEF14601824F0602624C1600BA9
:1059CA0024F670287F06127B6A8021127117801CC8
:1059DA007F06127B6A1274AE127632126FA5D265F6
:1059EA00800A7F06127B6A12672FD2653065AAE4A5
:1059FA00786CF6D2697F01125A2F7F01126BC17D32
:105A0A00467F021276B67D1E7F071276B67D147F18
:105A1A00081276B67D327F031276B6C2697F01120A
:045A2A005A2FC25CD1
:015A2E002255
:10672F00756701756500756620E4F5577F02127B6A
:10673F006AE5672402F559AF67127B6AE4F558E5FD
:10674F00662558F582E43565F583E0FF127B6AE52F
:10675F00662558F582E43565F583E02559F5590529
:10676F0058E558C3948040D7AF59127B6A7F031204
:10677F007B6A127B72EF641560160567748025665D
:10678F00F566E43565F5650557E557C39435409CC7
:01679F0022D7
:1074AE00756701756500756620E4F557127605500F
:1074BE00077F06127B6A80057F15027B6A0567745B
:1074CE00802566F566E43565F5650557E557C39481
:0374DE003540D95D
:0174E1002288
:10760500E4F558127B7274502558F582E4341CF564
:1076150083EFF00558E558C3948440E7127AA090AB
:0C7625001CD2E0B507051278D0D322C3B8
:017631002236
:1078D000E4FF74522FF582E4341CF583E0FEE56684
:0F78E0002FF582E43565F583EEF0000FBF80E3EE
:0178EF002276
:107AA000E4FFFE74502EF582E4341CF583E02FFFD2
:047AB0000EBE82EF95
:017AB40022AF
:10711700E4F557F55D755CE0755B93755A04F559B1
:10712700785974FF12595CE4FBFAF9F8C31259490C
:1071370050253098EB1200068F58E5586404601705
:10714700AF5D055D74502FF582E4341CF583E55877
:07715700F02557F55780C930
:01715E00220E
:04000600AF99C29854
:01000A0022D3
:087B6A003099FDC2998F9922A8
:077B72003098FDAF99C298A5
:017B790022E9
:105B970007010203040506070707060504030201B8
:105BA70003010A0A03020A0A03030A0A03040A0A88
:105BB700030307050303020503070A0A04024B0050
:105BC700040438072E03024B0004043802055F0063
:105BD7000302055F000402055F000502055F00067A
:105BE70002055F000702055F000802055F00090262
:105BF700055F000A02055F000B02055F000C020546
:105C07005F000D02055F000E02055F000F02055FD2
:105C1700001002055F001102055F001204072E083D
:105C2700260640033204072E082606400253080CB6
:075C37000A1D040000241BFC
:10001600C2AF9000207491F09000217481F090009E
:1000260022F0900023F09000247403F090002574D1
:10003600BFF09000267408F0900027740FF090002F
:10004600307409F0A37403F0E4A3F0A37410F0A3D2
:100056007403F0E4A3F0A37415F0A37403F0A3747F
:1000660015F0A37403F0E4A3F0A37410F0A37403D3
:10007600F0E4A3F0A37409F0A37403F0A37415F0DD
:10008600A37403F0A314F0A3741AF0A37403F0E4AA
:10009600A3F0A3F0A3F0A3741AF0A37403F0A314BF
:1000A600F0A37415F0A37403F0E4A3F0A3F0A3F097
:1000B6007E5B7FA77C007D807B041272327E5B7F35
:1000C600AB7C007D887B041272327E5B7FAF7C0046
:1000D6007D907B041272327E5B7FB37C007D987BC1
:1000E600041272327E5B7FBB7C007DA07B041272A1
:1000F600327E5B7FB77C007DA87B041272327E5B0A
:100106007FBF7C007DB07B041272327E5B7F977C62
:10011600007D707B081272327E5B7F9F7C007D784B
:100126007B081272327E5B7FC37C037D807B091263
:1001360072327E5B7FCC7C037DA07B071272327E9F
:100146005B7FD37C037DC07B051272327E5B7FD8DA
:100156007C037DE07B051272327E5B7FDD7C047D55
:10016600007B051272327E5B7FE27C047D207B057C
:100176001272327E5B7FE77C047D407B0512723211
:100186007E5B7FEC7C047D607B051272327E5B7F3A
:10019600F17C047D807B051272327E5B7FF67C04E7
:1001A6007DA07B051272327E5B7FFB7C047DC07B6B
:1001B600051272327E5C7F007C047DE07B05127244
:1001C600327E5C7F057C057D007B051272327E5C8B
:1001D6007F0A7C057D207B051272327E5C7F0F7C58
:1001E600057D407B051272327E5C7F147C057D6046
:1001F6007B051272327E5C7F197C057D807B051241
:1002060072327E5C7F1E7C057DA07B051272327E7B
:100216005C7F237C057DC07B091272327E5C7F2C5D
:100226007C057DE07B09127232900600E4F0A3742F
:10023600B4F0900602E4F0A374B4F0900604E4F07F
:10024600A374B4F0900606E4F0A374B4F090061814
:100256007401F0A374E0F090061AE4F0A37478F049
:1002660090061EE4F0A3743CF09006087402F0A316
:100276007458F090060A7402F0A37458F090060CB5
:100286007402F0A37458F090060E7402F0A374582A
:10029600F09006107401F0A3742CF090061274020C
:1002A600F0A37458F09006147403F0A37484F090CD
:1002B60006167404F0A374B0F07407900620F0A339
:1002C600F0900622F0A3F090061C7402F0A3745876
:1002D600F0900630740AF09006317428F0900633D8
:1002E600740AF0900634F09006327405F07E5C7F56
:1002F600357C067D407B0912723290063D7417F0FC
:1003060090063E740CF090063C7419F0E490063F9B
:10031600F090063B740CF09006527401F090073092
:100326007469F0A37411F09006537401F0900750AD
:100336007469F0A37410F09006547401F09007707D
:100346007469F0A37421F09006557401F09007903B
:100356007469F0A37420F09006567401F09007B00B
:100366007469F0A37431F09006577401F09007D0C9
:100376007469F0A37430F09006587401F09007F099
:100386007469F0A37441F09006597401F090081056
:100396007469F0A37440F090065A7401F090083026
:1003A6007462F0A37411F0A37432F0A37401F0A385
:1003B6007450F0A37410F090065B7401F09008502E
:1003C6007461F0A37420F0A37462F0A37411F0A317
:1003D6007432F0A37402F0A37450F0A37410F0907A
:1003E600065C7401F09008707451F0A37411F0A3C8
:1003F6007433F0A3E4F0A37451F0A37410F09006E4
:100406005D7401F09008907462F0A37411F0A37407
:1004160030F0A37402F0A37462F0A37410F0900697
:100426005E7401F09008B07451F0A37411F0A374D7
:1004360041F0A37410F0A37451F0A37410F0900669
:100446005F7401F09008D07451F0A37411F0A37496
:1004560034F0A37414F0A37451F0A37410F0900652
:10046600607401F09008F07451F0A37411F0A37455
:1004760034F0A37418F0A37451F0A37410F090062E
:10048600617401F09009107451F0A37411F0A37413
:1004960034F0A37428F0A37451F0A37410F09006FE
:1004A600627401F09009307462F0A37411F0A374C1
:1004B60030F0A37403F0A37462F0A37410F09006F6
:1004C600637401F09009507462F0A37411F0A37480
:1004D60030F0A37404F0A37462F0A37410F09006D5
:1004E600647401F09009707462F0A37411F0A3743F
:1004F60060F0A37401F0A37495F0A3743DF0A374A7
:1005060090F0A37401F0A37498F0A37426F0A3747A
:1005160096F0A37440F0A37462F0A37410F0A37471
:1005260061F0A37470F09006657401F09009907400
:1005360062F0A37411F0A37460F0A37401F0A374C5
:1005460095F0A3743DF0A37490F0A37401F0A37426
:1005560096F0A37438F0A37462F0A37410F09006BA
:10056600667401F09009B07462F0A37411F0A3747C
:1005760060F0A37401F0A37495F0A3743DF0A37426
:1005860090F0A37402F0A37498F0A37426F0A374F9
:1005960096F0A37440F0A37462F0A37410F0A374F1
:1005A60061F0A37470F09006677401F09009D0743E
:1005B60062F0A37411F0A37460F0A37401F0A37445
:1005C60095F0A3743DF0A37490F0A37402F0A374A5
:1005D60096F0A37438F0A37462F0A37410F090063A
:1005E600687401F09009F07462F0A37411F0A374BA
:1005F60060F0A37401F0A37495F0A3743DF0A374A6
:1006060090F0A37403F0A37498F0A37426F0A37477
:1006160096F0A37440F0A37462F0A37410F0A37470
:1006260061F0A37470F09006697401F0900A10747A
:1006360062F0A37411F0A37460F0A37401F0A374C4
:1006460095F0A3743DF0A37490F0A37403F0A37423
:1006560096F0A37438F0A37462F0A37410F09006B9
:100666006A7401F0900A307462F0A37411F0A374F6
:1006760060F0A37401F0A37495F0A3743DF0A37425
:1006860090F0A37404F0A37498F0A37426F0A374F6
:1006960096F0A37440F0A37462F0A37410F0A374F0
:1006A60061F0A37470F090066B7401F0900A5074B8
:1006B60062F0A37411F0A37460F0A37401F0A37444
:1006C60095F0A3743DF0A37490F0A37404F0A374A2
:1006D60096F0A37438F0A37462F0A37410F0900639
:1006E6006C7401F0900A707462F0A37411F0A37434
:1006F60060F0A37401F0A37430F0A37405F0A37442
:1007060062F0A37410F090066D7401F0900A907474
:1007160062F0A37421F0A37460F0A37401F0A374D3
:1007260030F0A37406F0A37462F0A37420F0900670
:100736006E7401F0900AB07462F0A37431F0A37481
:1007460060F0A37401F0A37430F0A37407F0A374EF
:1007560062F0A37430F090066F7401F0900AD074C2
:1007660062F0A37441F0A37460F0A37401F0A37463
:1007760030F0A37408F0A37462F0A37440F09006FE
:10078600707401F0900AF07464F0A37411F0A3740D
:1007960096F0A37432F0A37495F0A3741EF0A374BC
:1007A60098F0A3744BF0A37464F0A37410F0900651
:1007B600717401F0900B107464F0A37411F0A374BB
:1007C60096F0A37432F0A37495F0A3741EF0A3748C
:1007D60093F0A37418F0A37464F0A37410F0900659
:1007E600737401F0900B507462F0A37411F0A3744B
:1007F60060F0A37401F0A37495F0A3743DF0A374A4
:1008060090F0A37402F0A37497F0A37426F0A37477
:1008160093F0A37418F0A37462F0A37410F0A37499
:1008260070F0A37410F09006747401F0900B70745D
:1008360062F0A37411F0A37460F0A37401F0A374C2
:1008460095F0A3743DF0A37490F0A37403F0A37421
:1008560097F0A37426F0A37493F0A37418F0A3740E
:1008660062F0A37410F0A37470F0A37420F09006E5
:10087600757401F0900B907462F0A37411F0A37478
:1008860060F0A37401F0A37495F0A3743DF0A37413
:1008960090F0A37404F0A37497F0A37426F0A374E5
:1008A60093F0A37418F0A37462F0A37410F0A37409
:1008B60070F0A37430F09006817401F0900D1074FE
:1008C60062F0A37411F0A37460F0A37401F0A37432
:1008D60092F0A3744BF0A37490F0A37404F0A37485
:1008E60094F0A37438F07499A3F0A3F0A37460F0A5
:1008F600A37401F0A37462F0A37410F01222F8122C
:100906006FA5D2697F01125A2F7D2F7F071276B607
:100916007D0C7F031276B67D327F061276B67D1E7B
:100926007F051276B690001F7401F0FD7F1F7E00D2
:0B0936001272B3C2697F01125A2F2217
:1022F8009001007402F0A3740DF0A37402F090062C
:10230800A014F09010F07464F0A37411F0A3749703
:10231800F0A3742EF0A37495F0A3743DF0A3749009
:10232800F0A37402F0A37496F0A37438F0A3746455
:10233800F0A37410F0A37470F0A37411F090010866
:102348007402F0A3740EF0A37402F09006A114F0C6
:102358009011107461F0A37410F0A37464F0A37466
:1023680011F0A37497F0A3742EF0A37495F0A374DE
:102378003DF0A37490F0A37402F0A37496F0A374D4
:1023880036F0A37464F0A37410F0A37470F0A3740F
:1023980010F09001107402F0A3740DF0A37403F010
:1023A8009006A27401F09011307464F0A37411F0D7
:1023B800A37497F0A3742EF0A37495F0A3743DF062
:1023C800A37490F0A37403F0A37496F0A37438F088
:1023D800A37464F0A37410F0A37470F0A37421F0D4
:1023E8009001187402F0A3740EF0A37403F0900621
:1023F800A37401F09011507461F0A37410F0A374E9
:1024080064F0A37411F0A37497F0A3742EF0A3746E
:1024180095F0A3743DF0A37490F0A37403F0A37433
:1024280096F0A37436F0A37464F0A37410F0A37448
:1024380070F0A37420F09001207402F0A3740DF0E2
:10244800A37404F09006A47401F09011707464F001
:10245800A37411F0A37497F0A3742EF0A37495F0ED
:10246800A3743DF0A37490F0A37404F0A37496F0E1
:10247800A37438F0A37464F0A37410F0A37470F01C
:10248800A37431F09001287402F0A3740EF0A374C1
:1024980004F09006A57401F09011907461F0A37493
:1024A80010F0A37464F0A37411F0A37497F0A374EC
:1024B8002EF0A37495F0A3743DF0A37490F0A37468
:1024C80004F0A37496F0A37436F0A37464F0A374B4
:1024D80010F0A37470F0A37430F09001307403F01E
:1024E800A3740DF0A37402F0A304F09006A674017F
:1024F800F09011B07464F0A37411F0A37497F0A372
:10250800742EF0A37495F0A3743DF0A37490F0A317
:102518007402F0A37490F0A37403F0A37496F0A36C
:102528007438F0A37464F0A37410F0A37470F0A36B
:102538007441F09001387403F0A3740EF0A3740290
:10254800F0A304F09006A77401F09011D07461F024
:10255800A37410F0A37464F0A37411F0A37497F03B
:10256800A3742EF0A37495F0A3743DF0A37490F0B7
:10257800A37402F0A37490F0A37403F0A37496F00C
:10258800A37436F0A37464F0A37410F0A37470F00D
:10259800A37440F09001407404F0A3740DF0A37488
:1025A80002F0A304F0A304F09006A87401F09011BF
:1025B800F07464F0A37411F0A37497F0A3742EF070
:1025C800A37495F0A3743DF0A37490F0A37402F083
:1025D800A37490F0A37403F0A37490F0A37404F0B0
:1025E800A37496F0A37438F0A37464F0A37410F085
:1025F800A37470F0A37441F0A37470F0A37451F045
:102608009001487404F0A3740EF0A37402F0A304BC
:10261800F0A304F09006A97401F09012107461F010
:10262800A37410F0A37464F0A37411F0A37497F06A
:10263800A3742EF0A37495F0A3743DF0A37490F0E6
:10264800A37402F0A37490F0A37403F0A37490F041
:10265800A37404F0A37496F0A37436F0A37464F022
:10266800A37410F0A37470F0A37440F0A37470F016
:05267800A37450F022E4
:0A7232008E4C8F4D8C4E8D4F8B500B
:10723C00E4F9C3E5506480F8E96480985028E9FFCC
:10724C003395E0FEE54D2FF582E54C3EF583E49356
:10725C00FFE9FD3395E0FCE54F2DF582E54E3CF55D
:06726C0083EFF00980CC65
:0172720022F9
:107A1200D291C2A4C2A5C2A6C2A7007F05127A8AC9
:097A220000127A7400D2A7D2917F
:017A2B002238
:10792F00127A12EF20E0F9D291C2A4C2A5C2A6C268
:0E793F00A7007F06127A8A0000D2A7D29122FA
:10794D00127A12EF20E0F9D291C2A4C2A5C2A6C24A
:0E795D00A7007F04127A8A0000D2A7D29122DE
:046E11008E528F53BB
:106E1500AE04AF058E568F57D291C2A4C2A5C2A6A5
:106E2500C2A7007F03127A8AE552FF127A8AAF530E
:106E3500127A8AE4F554F555127A74E5572555F515
:106E450082E5563554F583EFF00555E55570020595
:0E6E550054C39420E554940040DED2A7D2919D
:016E6300220C
:0868DE008E5D8F5E8C5F8D6002
:1068E600127A12EF20E0F912792F855D63855E64D6
:1068F600D291C2A4C2A5C2A6C2A7007F02127A8AFA
:10690600E55FFF127A8AAF60127A8AE4F561F56272
:10691600E5642562F582E5633561F583E0FF127A69
:106926008A0562E56270020561C39420E561940000
:0769360040DE00D2A7D29160
:01693D002237
:0A67A0008E4C8F4D8C4E8D4F8B50A8
:1067AA00C2AF12792F127A12EF20E0F9854E528584
:1067BA004F53D291C2A4C2A5C2A6C2A7007F021299
:1067CA007A8AE54CFF127A8AAF4D127A8AE4F55139
:1067DA00AF50EF3395E0FEC3E5519FEE6480F87445
:1067EA0080985014E5532551F582E43552F583E03B
:1067FA00FF127A8A055180D800D2A7D29112794D18
:02680A00D2AF0B
:01680C002269
:1072B3008E5B8F5C8D5DC2AF12792F127A12EF2035
:1072C300E0F9D291C2A4C2A5C2A6C2A7007F02124E
:1072D3007A8AE55BFF127A8AAF5C127A8AAF5D1213
:0E72E3007A8A0000D2A7D29112794DD2AF2242
:0477F9008E4C8F4DD6
:1077FD00D291C2A4C2A5C2A6C2A77F03127A8AE5FE
:10780D004CFF127A8AAF4D127A8A127A74D2A7D2AD
:01781D0091D9
:01781E002247
:10715F00C2AF754E00754F20755000755120E4F584
:10716F004CF54DAD4FAC4EAF51AE50126E11742069
:10717F00254FF54FE4354EF54E74202551F551E46A
:10718F003550F550054DE54D7002054CC394D6E5CD
:07719F004C940040CED2AF7A
:0171A60022C6
:106FA500C2AF755B00755C20755900755A20E4F514
:106FB50057F558AD5AAC59AF5CAE5B1268DE74201C
:106FC500255AF55AE43559F5597420255CF55CE4E4
:106FD500355BF55B0558E55870020557C394D6E552
:0A6FE50057940040CE12794DD2AF50
:016FEF00227F
:046EB6008C4D8D4E24
:106EBA00EF6048D22BD22CD22DD22EE4F54F854E3C
:106ECA0082854D83E0FEA3E04E6028AF4FEF3395F5
:106EDA00E0FEEF25E0FFEE33FEE54E2FF582E54DAD
:106EEA001254DD926520650B054FC3E54F6480940B
:0B6EFA009040CBC22BC22CC22DC22E38
:016F05002269
:047273008C4D8D4E63
:10727700EF6038E4F54F854E82854D83E0FEA3E04D
:107287004E6028AF4FEF3395E0FEEF25E0FFEE337A
:10729700FEE54E2FF582E54D1254DD926520650B14
:0B72A700054FC3E54F6480949040CB7E
:0172B20022B9
:0854DD003EF583E0FEA3E0FFB1
:0454E500AD07AC065D
:1054E900C266780CEF088006A2E0CE13CE13D8F876
:1054F900540FF5507808AF05AE04EF088006A2E016
:10550900CE13CE13D8F8540FF5517804AF05AE0475
:10551900EF088006A2E0CE13CE13D8F8540FF55247
:10552900ED540FF553E550607CB4010BAB53AD520C
:10553900AF51125804806EE550B4030BAB53AD5212
:10554900AF51126A59805EE550B4040BAB53AD52AA
:10555900AF51126AB4804EE550B4050BAB53AD524E
:10556900AF51123CE8803EE550B4060BAB53AD5247
:10557900AF5112180F802EE550B4070BAB53AD5243
:10558900AF51125408801EE550B4080BAB53AD520D
:10559900AF51126E64800EE550B40909AB53AD5298
:0755A900AF51127844A26625
:0155B00022D8
:105804008F548D558B56E554B40113900020E0FF5E
:10581400126A01900020EFF0FD7F2002589FE554AA
:10582400B402119000211269FB900021EFF0FD7F7A
:105834002102589FE554B403109000221269FB9092
:105844000022EFF0FD7F228052E554B40410900052
:10585400231269FB900023EFF0FD7F23803DE55484
:10586400B405109000241269FB900024EFF0FD7F32
:10587400248028E554B406109000251269FB90009A
:1058840025EFF0FD7F258013E554B407139000261F
:105894001269FB900026EFF0FD7F267E000272B3B2
:1058A400E554B408169000271269FB900027EFF026
:0C58B400FD7F277E001272B312763222B4
:0669FB00E0FFAB56AD55B4
:106A0100D267AC07BD01047E018033BD02047E0262
:106A1100802CBD03047E048025BD04047E08801EF5
:106A2100BD05047E108017BD06047E208010BD07C1
:106A3100047E408009BD08047E808002C267BB01DC
:106A410005EE4204800BEB7006EEF452048002C2A4
:076A510067306703AF042268
:016A5800221B
:106A59008F548D558B56E554700BAD56AF55127B3F
:106A69001CE4FD801EE554B4010BAD56AF55127BF5
:106A79001C7D01800EE554B4020CAD56AF55127B56
:106A89001C7D0202385DE554B4030AE5557006120F
:106A990073A3C25822E554B40410AD56AF5512661B
:0B6AA900FD8F3F753D05E53D70FC22B0
:106AB4008F548D558B56E5547036E555B40108E571
:106AC4005614FF7D018026E555B40208E55614FFEF
:106AD4007D028019E555B40308E55614FF7D038053
:106AE4000CE55564047022E55614FF7D040271A779
:106AF400E554B40114E555D39400400DE5559405CF
:0A6B04005007753D01E53D70FC22CD
:103CE8008B54EF7017BD0114E5547002C220E554DF
:103CF80064016003023E54D220023E54EF7017BDA7
:103D08000214E5547002C221E55464016003023EC6
:103D180054D221023E54EF7017BD0314E5547002CB
:103D2800C222E55464016003023E54D222023E548A
:103D3800EF7017BD0414E5547002C223E554640102
:103D48006003023E54D223023E54EF701BBD051897
:103D5800E5547004C220C221E55464016003023EA8
:103D680054D220D221023E54EF701BBD0618E554F0
:103D78007004C222C223E55464016003023E54D297
:103D880022D223023E54BF0117BD0114E55470022C
:103D9800C224E55464016003023E54D224023E5416
:103DA800BF0117BD0214E5547002C225E554640131
:103DB8006003023E54D225023E54BF0116BD0313D0
:103DC800E5547002C226E55464016003023E54D2F1
:103DD800268079BF0113BD0410E5547002C227E59F
:103DE8005464017067D2278063BF0117BD0514E5CD
:103DF800547004C224C225E5546401704FD224D201
:103E0800258049BF0117BD0614E5547004C226C2B7
:103E180027E55464017035D226D227802FEF64013C
:103E2800702AED64097025E554B401047F018019F6
:103E3800E554B402047F028010E554B403047F0300
:103E48008007E554B404057F04126BC17F327E00FD
:043E58001279DD22DC
:10180F008F548D558B56E5547016AD56AF55127BD0
:10181F001C901D14EFF0901D14E0D3940050F7228C
:10182F00E554B40117E555B40112E5567002C2082C
:10183F00E55664016003021BB5D20822E554B401DA
:10184F0017E555B40212E5567002C209E556640158
:10185F006003021BB5D20922E554B40117E555B454
:10186F000312E5567002C20EE55664016003021BB7
:10187F00B5D20E22E554B40117E555B40412E5565E
:10188F007002C20CE55664016003021BB5D20C2234
:10189F00E554B4011BE555B40516E5567004C208AE
:1018AF00C209E55664016003021BB5D208D20922B2
:1018BF00E554B40118E555B40613E5567004C20E8D
:1018CF00C20CE55664016003021BB58024E5546425
:1018DF00017023E555B4071EE5567008C208C2090A
:1018EF00C20EC20CE55664016003021BB5D208D2CA
:1018FF0009D20ED20C22E554B4021DE555B40118DD
:10190F00E5567004C208C220E55664016003021B4D
:10191F00B5D208D220021AD5E554B4021DE555B44C
:10192F000218E5567004C209C221E556640160032E
:10193F00021BB5D209D221021A61E554B4021DE58A
:10194F0055B40318E5567004C20EC222E556640161
:10195F006003021BB5D20ED222021A85E554B402DF
:10196F001DE555B40418E5567004C20CC223E556A4
:10197F0064016003021BB5D20CD223021AA8E554EE
:10198F0064027026E55564057020E5567008C2089C
:10199F00C209C220C221E55664016003021BB5D201
:1019AF0008D209D220D221021AD5E554640270263A
:1019BF00E55564067020E5567008C20EC20CC222AF
:1019CF00C223E55664016003021BB5D20ED20CD2BE
:1019DF0022D223021A85E55464027035E555640757
:1019EF00702FE5567010C208C209C20EC20CC22079
:1019FF00C221C222C223E55664016003021BB5D285
:101A0F0008D209D20ED20CD220D221D222D22380D8
:101A1F0065E554B4031DE555B40118E5567004C2CD
:101A2F0008C224E55664016003021BB5D208D22414
:101A3F00021AD5E554B4031FE555B4021AE55670E2
:101A4F0004C209C225E55664016003021BB5D20921
:101A5F00D2257F02021B04E554B4031EE555B403DF
:101A6F0019E5567004C20EC226E5566401600302E2
:101A7F001BB5D20ED2267F03807BE554B4031EE53F
:101A8F0055B40419E5567004C20CC227E55664011B
:101A9F006003021BB5D20CD2277F048058E5546433
:101AAF00037027E55564057021E5567008C208C21A
:101ABF0009C224C225E55664016003021BB5D20892
:101ACF00D209D224D2257F01802BE55464037028DC
:101ADF00E55564067022E5567008C20EC20CC22688
:101AEF00C227E55664016003021BB5D20ED20CD299
:101AFF0026D2277F03026BC1E554B4040AE555B41F
:101B0F000105AF560265C3E554B4040AE555B402A6
:101B1F0005AF56026876E5546409701EE555B401A9
:101B2F0019E5567003C20A22E556B40103D20A2200
:101B3F00E556640270707F058069E5546409701E74
:101B4F00E555B40219E5567003C20B22E556B401F0
:101B5F0003D20B22E5566402704C7F068045E55494
:101B6F006409701EE555B40319E5567003C20F22C0
:101B7F00E556B40103D20F22E556640270287F07A1
:101B8F008021E5546409701EE555B40419E55670BB
:101B9F0003C20D22E556B40103D20D22E556B4025D
:071BAF00057F08125FEC2224
:10540800AC07EC60030254BEBD010CEB70099000C0
:105418001FE054FDF0800DBD010ABB010790001F7D
:10542800E04403F0BD020CEB700990001FE054FB50
:10543800F0800DBD020ABB010790001FE04405F093
:10544800BD030CEB700990001FE054F7F0800DBD10
:10545800030ABB010790001FE04409F0BD040CEBF0
:10546800700990001FE054F9F0800DBD040ABB01DB
:105478000790001FE04407F0BD050CEB7009900091
:105488001FE054F3F0800DBD050ABB010790001F13
:10549800E0440DF0BD060CEB700990001FE054F1DC
:1054A800F08025ED64067020EB6401701B90001FEE
:1054B800E0440FF08012BC010FED700CEB7004C2D9
:1054C800298005BB0102D22990001FE0FD7F1F7EC5
:0554D800001272B32276
:106E64008F548D558B56E554700C127B18744F2F2C
:106E7400F58274068020E554B4010C127B18744F1B
:106E84002FF58274068024E554B40210127B187422
:106E94009F2FF58274063EF583E4F022E554B40393
:106EA40010127B18749F2FF58274063EF5837401CB
:026EB400F022CA
:027844008F545F
:10784600AF057804EF08800123D8FD4BF555E554C4
:10785600B40908E555B49903025F56AD55AF541205
:0278660076B6F4
:0178680022FD
:1065C300E545B40109BF0106D220D2088060E54544
:1065D300B40109EF7006C220C2088052E545B40237
:1065E30009BF0106D221D2098044E545B40209EF6F
:1065F3007006C221C2098036E545B40309BF01060E
:10660300D222D20E8028E545B40309EF7006C222D8
:10661300C20E801AE545B40409BF0106D223D20C89
:10662300800CE545B40407EF7004C223C20C127951
:0A663300C1AF3E126BC11279A5221F
:10687600E545B40108BF0105D224D20822E545B496
:106886000108EF7005C224C20822E545B40208BF1C
:106896000105D225D20922E545B40208EF7005C2EA
:1068A60025C20922E545B40308BF0105D226D20E4A
:1068B60022E545B40308EF7005C226C20E22E5455F
:1068C600B40408BF0105D227D20C22E545B404075B
:0868D600EF7004C227C20C227E
:047B1800AD56AF5562
:0D7B1C00EF75F00AA47C002DFFEC35F0FEA3
:017B29002239
:020941008F4DD8
:10094300C266E4F53DD25CD269125A2F7D4B7F0219
:100953001276B67D04E4FF1276B67D387F041276F4
:10096300B67D607F021276B690061CE0FFA3E0908E
:100973001CE8CFF0A3EFF0C269AF4D125A2FE4F594
:1009830046C208123346E54DB40106A2499265807A
:100993001FE54DB40206A24D92658014E54DB403E4
:1009A30006A25192658009E54DB40404A2549265F0
:1009B300901CE8E07002A3E07005D266020F8B3052
:1009C30065C1123346E54DB40106A2499265801F05
:1009D300E54DB40206A24D92658014E54DB40306BD
:1009E300A25192658009E54DB40404A25492652096
:1009F30065D0E54DB4010A754E1B754F10786880BC
:100A03002BE54DB4020A754E1B754F607869801C47
:100A1300E54DB4030A754E1B754FB0786A800DE53A
:100A23004DB4040B754E1C754F00786BE6F550E51D
:100A330050D394005003020F85854F82854E83E087
:100A4300640B6003020F80A3E0FFB40A0AE550B40D
:100A53000205D266020F85EF64017032854F8285ED
:100A63004E83A3A3E064037025E550B40520854FAE
:100A730082854E83A3A3A3E0FFE54F2404F582E41C
:100A8300354EF583E0FDAB4D123FB6020F85854F22
:100A930082854E83A3E0B40121854F82854E83A3D3
:100AA300A3E0B40415E550D39405400EAB4DAD4F10
:100AB300AC4EAF5012350C020F85854F82854E83A5
:100AC300A3E064017032854F82854E83A3A3E06463
:100AD300057025E550B40520854F82854E83A3A379
:100AE300A3E0FFE54F2404F582E4354EF583E0FDF2
:100AF300AB4D126543020F85854F82854E83A3E07C
:100B030064017032854F82854E83A3A3E06406702F
:100B130025E550B40520854F82854E83A3A3A3E02A
:100B2300FFE54F2404F582E4354EF583E0FDAB4D3C
:100B3300125C3E020F85854F82854E83A3E0B4018C
:100B430021854F82854E83A3A3E0B40715E550D3D7
:100B53009405400EAB4DAD4FAC4EAF50124CA702B7
:100B63000F85854F82854E83A3E064017032854FE4
:100B730082854E83A3A3E064087025E550B4052065
:100B8300854F82854E83A3A3A3E0FFE54F2404F59D
:100B930082E4354EF583E0FDAB4D126B0E020F85FB
:100BA300854F82854E83A3E0B40219854F82854E1B
:100BB30083A3A3E0B4080DE550B40308AF4D127648
:100BC3008A020F85854F82854E83A3E064027024D9
:100BD300854F82854E83A3A3E0B40818E550B4047F
:100BE30013854F82854E83A3A3A3E0FFAD4D1277F8
:100BF30083020F85854F82854E83A3E0B402198556
:100C03004F82854E83A3A3E0B4090DE550B40308D6
:100C1300AF4D12765E020F85854F82854E83A3E02A
:100C230064027024854F82854E83A3A3E0B4091820
:100C3300E550B40413854F82854E83A3A3A3E0FF3D
:100C4300AD4D12775B020F85854F82854E83A3E0FE
:100C530064037036854F82854E83A3A3E0640A70D4
:100C630029E55064057023854F82854E83A3A3A392
:100C7300E0FFE54F2404F582E4354EF583E0FD12F1
:100C83007976AD4D125745020F85854F82854E8388
:100C9300A3E06403703E854F82854E83A3A3E06483
:100CA300017031E550D39405402A854F82854E83E8
:100CB300A3A3A3E0FFE54F2404F582E4354EF583B7
:100CC300E0FD127976854D55AB50AD4FAC4E1246D3
:100CD3006A020F85854F82854E83A3E064037036D5
:100CE300854F82854E83A3A3E064027029E5506497
:100CF300057023854F82854E83A3A3A3E0FFE54FB1
:100D03002404F582E4354EF583E0FD127976AD4D8A
:100D1300127085020F85854F82854E83A3E0B4034D
:100D230019854F82854E83A3A3E0B4030DE550B428
:100D33000308AF4D1272F1020F85854F82854E83F2
:100D4300A3E0B40321854F82854E83A3A3E0B404BB
:100D530015E550D39403400EAB4DAD50AF4FAE4E9F
:100D6300125E25020F85854F82854E83A3E0B4036F
:100D730019854F82854E83A3A3E0B4050DE550B4D6
:100D83000308AF4D127B2A020F85854F82854E8360
:100D9300A3E0B4031D854F82854E83A3A3E0B4066D
:100DA30011E550B4050CAD4DAF4FAE4E12736A0250
:100DB3000F85854F82854E83A3E064037024854F9E
:100DC30082854E83A3A3E0B40718E550B4041385CA
:100DD3004F82854E83A3A3A3E0FFAD4D1278F002AB
:100DE3000F85854F82854E83A3E0B4031D854F8213
:100DF300854E83A3A3E0B40811E550B4050CAD4DB3
:100E0300AF4FAE4E127578020F85854F82854E83A4
:100E1300A3E064057022E550B4041D854F82854E1E
:100E230083A3A3E0FF854F82854E83A3A3A3E0FDA5
:100E3300AB4D122D80020F85854F82854E83A3E033
:100E4300B40524E54F2404F582E4354EF583E0B47C
:100E53000B15E550D39405400EAB4DAD50AF4FAEDF
:100E63004E12477A020F85854F82854E83A3E06435
:100E7300067022E550B4041D854F82854E83A3A3DB
:100E8300E0FF854F82854E83A3A3A3E0FDAB4D1204
:100E9300267D020F85854F82854E83A3E0B4062409
:100EA300E54F2404F582E4354EF583E0B40B15E5F4
:100EB30050D39405400EAB4DAD50AF4FAE4E1231F3
:100EC3005E020F85854F82854E83A3E064097022FD
:100ED300854F82854E83A3A3E0B40A16E550B4047C
:100EE30011854F82854E83A3A3A3E0FF126FF00207
:100EF3000F85854F82854E83A3E064097023854F58
:100F030082854E83A3A3E0B40117E550B404128590
:100F13004F82854E83A3A3A3E0FFAD4D125681807C
:100F230061854F82854E83A3E0B40920854F828576
:100F33004E83A3A3E0B40214E550D39404400DAB55
:100F430050AD4DAF4FAE4E1214648036854F82853F
:100F53004E83A3E064097025854F82854E83A3A346
:100F6300E0B40317E550B40412854F82854E83A382
:100F7300A3A3E0FFAD4D126F0680078000AF4D12B3
:100F83007988206603020986C258D269AF4D125A86
:100F93002F7D607F021276B67D327F031276B6C252
:0F0FA30069AF4D125A2F126FA5E4786CF6C25C3D
:010FB200221C
:08350C008F518C528D538B543A
:10351400855382855283A3A3A3E0FF8D828C83E528
:103524008224041266F48F55E555D39400500302A7
:1035340036ADE555942940030236ADE55164067075
:103544004FD269AF54125A2F7D527F051276B6AF0F
:1035540055124BA5E5532405F582E43552F583E075
:10356400B40112749F2555F582E43406F583740181
:10357400F07D38800F749F2555F582E43406F58379
:10358400E4F07D367F061276B6C269AF54025A2F34
:10359400E5532406F582E43552F583E0640B6003B9
:1035A4000236ADE5532405F582E43552F583E0B4E3
:1035B4000110749F2555F582E43406F5837401F0F7
:1035C400800D749F2555F582E43406F583E4F0E418
:1035D400FFFEE5532407F582E43552F583E5822E98
:1035E400F582E43583F583E0B40B04AF0680040E62
:1035F400BE08DFEF70030236ADC394084003023601
:10360400AD75F008E555A424F8F582E5F03400F52D
:1036140083EFF07E01EF2401FDE433FCEEC39DEC67
:103624006480F87480985036E5532406F582E435B6
:1036340052F583E5822EF582E43583F583E0FD754A
:10364400F008E555A424F8F582E5F03400F583E5A7
:10365400822EF582E43583F583EDF00E80B7E553D1
:103664002408F582E43552F583E5822FF582E435AA
:1036740083F583E0640B602DEF2408FEC3E5519EBF
:10368400F55175F0041258C0AEF0EE701CE55324E9
:1036940007FDE43552FC7E00ED2FFBEE3CFAAD5500
:1036A4007F011239E6D2688002C268AF54127B5C93
:0136B40022F3
:10788D008E5CF55DAF5BEF3395E0FEE5592FF5822C
:08789D00E5583EF583A3E0FF6E
:0A78A500EFD3940940037F00222274
:0839E6008F568D578A588B594A
:1039EE00755B01E4F55AAF5BEF3395E0FEE5592FB9
:1039FE00F582E5583EF583E0FF640970651278A5FF
:103A0E00755C008F5DAE5C7804EF08800633CE33B4
:103A1E00CE92E0D8F812788DEF425DAE5CAF5D7855
:103A2E0008EF08800633CE33CE92E0D8F88E5CF5E0
:103A3E005DAF5BEF3395E0FEE5592FF582E5583E1D
:103A4E00F583A3A3E0FFE55BFD3395E0FCE5592D7F
:103A5E00F582E5583CF583A3A3A3E0FD1279760227
:103A6E003B01AF5BEF3395E0FEE5592FF582E5584C
:103A7E003EF583E0FF1278A5755C008F5DAE5C7835
:103A8E0004EF08800633CE33CE92E0D8F812788D4C
:103A9E00EF425DAE5CAF5D7804EF08800633CE3347
:103AAE00CE92E0D8F88E5CF55DAF5BEF3395E0FE1D
:103ABE00E5592FF582E5583EF583A3A3E0FF127872
:103ACE00A5EF425DAE5CAF5D7804EF08800633CEA5
:103ADE0033CE92E0D8F88E5CF55DAF5BEF3395E0B8
:103AEE00FEE5592FF582E5583EF583A3A3A3E0FF2B
:103AFE001278A5EF425DE556701EAF5AEF3395E092
:103B0E00FEEF25E0FFEE33FE75F020E557A424D03E
:103B1E00F582E5F034068021E556B4012FAF5AEF59
:103B2E003395E0FEEF25E0FFEE33FE75F020E5570E
:103B3E00A424D0F582E5F03410F583E5822FF582CA
:103B4E00E5833EF583E55CF0A3E55DF07404255B4B
:103B5E00F55B055AC3E55A6480949050030239F41C
:013B6E002234
:084CA7008F518C528D538B5488
:104CAF00855382855283A3A3A3E0FF8D828C83E576
:104CBF008224041266F48F55E555D39400500302F5
:104CCF004D94E55594334003024D94E551640670BD
:104CDF004FD269AF54125A2F7D527F051276B6AF5D
:104CEF0055124BA5E5532405F582E43552F583E0C3
:104CFF00B40112744F2555F582E43406F58374011F
:104D0F00F07D38800F744F2555F582E43406F58316
:104D1F00E4F07D367F061276B6C269AF54025A2F81
:104D2F00E5532406F582E43552F583E0640B7055A4
:104D3F00E5532405F582E43552F583E0B401107490
:104D4F004F2555F582E43406F5837401F0800D7418
:104D5F004F2555F582E43406F583E4F074F92551B7
:104D6F00F55175F0041258C0AFF0EF7014E55324ED
:104D7F0006FBE43552FAAD55E4FF1239E6D26880EE
:104D8F000DC2688009C269AF54125A2FC268AF545E
:034D9F00127B5C28
:014DA20022EE
:023FB6008B512D
:103FB8001266FD8F54E554D3940050030240FAE58D
:103FC80054943340030240FAD269AF51125A2F7DFC
:103FD800527F051276B6AF54124BA5749F2554F53F
:103FE80082E43406F583E060047D3880027D367F04
:103FF800061276B67F2C7E011279DD75F008E5543D
:10400800A424F8F582E5F03400F583E0F552700752
:104018007D1B7F061276B67D577F021276B6E55273
:1040280070030240AB755301AF52EF3395E0FEEFDA
:104038002401FFE43EFEAD53ED3395E0FCC3ED9F54
:10404800EE6480F8EC6480985059AF53EF3395E0F4
:10405800FE75F008E554A424F8F582E5F03400F57F
:1040680083E5822FF582E5833EF583E0FFD394094B
:1040780040051271ED8028AF53EF3395E0FE75F0DF
:1040880008E554A424F8F582E5F03400F583E582C8
:104098002FF582E5833EF583E0FDE4FF1276B60551
:1040A8005380857F2C7E011279DD75F020E554A4BC
:1040B80024D0F582E5F03410F583E0FEA3E0FF900C
:1040C8000000EEF0A3EFF04E70077D1B7F0612761E
:1040D800B67D0C7F031276B6900000E07002A3E074
:1040E8006009E55414FD7F01122F74C269AF5102B3
:0940F8005A2FC268AF51127B5C23
:01410100229B
:042F74008F558D5692
:102F7800E4F557E555600302301FAF57EF3395E08E
:102F8800FEEF25E0FDEE33FCAF56EF3395E0FEEFA4
:102F98007805C333CE33CED8F924F0F58274063ED3
:102FA800F583E5822DF582E5833CF583E0FAA3E01D
:102FB800FB780CFFAE02088006A2E0CE13CE13D831
:102FC800F8540FF5587808AF03AE02EF088006A250
:102FD800E0CE13CE13D8F8540FF559AF56EF33950A
:102FE800E0FEEF7805C333CE33CED8F924F0F5826E
:102FF80074063EF583E5822DF582E5833CF583E092
:10300800FCA3E0FD7804FFAE04088006A2E0CE131E
:10301800CE13D8F80230C2E555640160030230CB04
:10302800AF57EF3395E0FEEF25E0FDEE33FCAF56EA
:10303800EF3395E0FEEF7805C333CE33CED8F924CD
:10304800F0F58274103EF583E5822DF582E5833C28
:10305800F583E0FAA3E0FB780CFFAE02088006A235
:10306800E0CE13CE13D8F8540FF5587808AF03AE56
:1030780002EF088006A2E0CE13CE13D8F8540FF55D
:1030880059AF56EF3395E0FEEF7805C333CE33CE14
:10309800D8F924F0F58274103EF583E5822DF58287
:1030A800E5833CF583E0FCA3E0FD7804FFAE04086B
:1030B8008006A2E0CE13CE13D8F8540FF55AED547B
:1030C8000FF55BE558700FE559700BE55A7007E589
:1030D8005B700302315DAD58E4FF1276B6AD59E47A
:1030E800FF1276B6E55864097048855A5CAF5CFEF5
:1030F8007804EF08800633CE33CE92E0D8F8F55C3A
:10310800E55B425CE55CB4990B7D09E4FF1276B699
:103118007D098027E55C75F00A84F55DFDE4FF1202
:1031280076B6E55D75F00AA4FFC3E55C9FF55DFD25
:103138008009AD5AE4FF1276B6AD5BE4FF1276B6AD
:103148007FF47E011279DD0557C3E557648094A0AA
:053158005003022F7B73
:01315D00224F
:025C3E008B5188
:105C40001266FD8F52E552D394005003025CDAE5F0
:105C50005294334003025CDAD269AF51125A2F7D5D
:105C6000527F051276B6AF52124BA5744F2552F5EE
:105C700082E43406F583E060047D3880027D367F5F
:105C8000061276B67F2C7E011279DD7F2C7E011202
:105C900079DD75F020E552A424D0F582E5F03406D4
:105CA000F583E0FEA3E0FF900000EEF0A3EFF04EDE
:105CB00070077D1B7F061276B67D0C7F031276B6C9
:105CC000900000E07002A3E06009E55214FDE4FFDB
:105CD000122F74C269AF51025A2FC268AF51127BA2
:015CE0005C67
:015CE10022A0
:026543008B517A
:106545001266FDAD07EDD39400406BED94335066B4
:10655500E4FCECFF3395E0FEEF25E0FFEE33FE753E
:10656500F020EDA424D0F582E5F03410F583E58222
:106575002FF582E5833EF583E4F0A3F00CBC10D241
:10658500749F2DF582E43406F583E4F0FCECFF33CB
:1065950095E0FE75F008EDA424F8F582E5F03400E9
:1065A500F583E5822FF582E5833EF583E4F00CBCA7
:0D65B50008DBD2688002C268AF51127B5C27
:0165C20022B6
:026B0E008B51A9
:106B10001266FDAD07EDD394004045ED943350402F
:106B2000E4FCECFF3395E0FEEF25E0FFEE33FE756D
:106B3000F020EDA424D0F582E5F03406F583E5825B
:106B40002FF582E5833EF583E4F0A3F00CBC10D270
:106B5000744F2DF582E43406F583E4F0D2688002A8
:076B6000C268AF51127B5C1B
:016B6700220B
:1074E2002430F58274003EF583EDF0AF55EF33950D
:1074F200E0FEE5522FF582E5513EF583A3A3E0FFBE
:10750200D3EF648094814008EF6480948A50012212
:037512007F0022D5
:107B0500D3EF648094804008EF648094A1500122F3
:037B15007F0022CC
:081464008E518F528D538B5401
:10146C008F828E83A3A3A3E014F55674FC2554F548
:10147C00546403600FE55464076009E554640B6021
:10148C0003021807C3E556648094805003021807C2
:10149C00E556648094884003021807E4F555AF566E
:1014AC00EF3395E0FEEF7803C333CE33CED8F92477
:1014BC0030F58274003EF583AF55EF3395E0FEE5D1
:1014CC00822FF582E5833EF583E4F00555E555B4AE
:1014DC0008CC755504E5546403705FAF55EF339534
:1014EC00E0FEE5522FF582E5513EF583E0FFE55530
:1014FC00FD3395E0FCE5522DF582E5513CF583A3D7
:10150C00E0FD1266FD127B05AD07AF56EF3395E09B
:10151C00FEEF7803C333CE33CED8F91274E2AD07A5
:10152C00AF56EF3395E0FEEF7803C333CE33CED80E
:10153C00F92431F58274000217FEE5546407600348
:10154C00021639AF55EF3395E0FEE5522FF582E5E3
:10155C00513EF583E0FFE555FD3395E0FCE5522D5A
:10156C00F582E5513CF583A3E0FD1266FD127B0587
:10157C00AD07AF56EF3395E0FEEF7803C333CE33B0
:10158C00CED8F91274E2AD07AF56EF3395E0FEEF0B
:10159C007803C333CE33CED8F92431F58274003EB0
:1015AC00F583EDF0AF55EF3395E0FEE5522FF58264
:1015BC00E5513EF583A31274FEAD07AF56EF33959C
:1015CC00E0FEEF7803C333CE33CED8F91266B612F1
:1015DC007B05AD07AF56EF3395E0FEEF7803C333D1
:1015EC00CE33CED8F92433F58274003EF583EDF07A
:1015FC00AF55EF3395E0FEE5522FF582E5513EF500
:10160C0083E5822406F582E43583F583E0FF1275C9
:10161C0002AD07AF56EF3395E0FEEF7803C333CE40
:10162C0033CED8F92434F58274000217FEE55464E5
:10163C000B6003021807AF55EF3395E0FEE5522F10
:10164C00F582E5513EF583E0FFE555FD3395E0FC71
:10165C00E5522DF582E5513CF583A3E0FD1266FDC4
:10166C00127B05AD07AF56EF3395E0FEEF7803C361
:10167C0033CE33CED8F91274E2AD07AF56EF3395B3
:10168C00E0FEEF7803C333CE33CED8F92431F582A4
:10169C0074003EF583EDF0AF55EF3395E0FEE55267
:1016AC002FF582E5513EF583A31274FEAD07AF56BC
:1016BC00EF3395E0FEEF7803C333CE33CED8F91277
:1016CC0066B6127B05AD07AF56EF3395E0FEEF78AB
:1016DC0003C333CE33CED8F92433F58274003EF5F0
:1016EC0083EDF0AF55EF3395E0FEE5522FF582E533
:1016FC00513EF583E5822406F582E43583F583E0DB
:10170C00FF127502AD07AF56EF3395E0FEEF78038D
:10171C00C333CE33CED8F92434F58274003EF5832E
:10172C00EDF0AF55EF3395E0FEE5522FF582E55124
:10173C003EF583E5822407F582E43583F583E0FFEB
:10174C00127502AD07AF56EF3395E0FEEF7803C389
:10175C0033CE33CED8F92435F58274003EF583EDC3
:10176C00F0AF55EF3395E0FEE5522FF582E5513E93
:10177C00F583E5822408F582E43583F583E0FFE503
:10178C0055FD3395E0FCE5522DF582E5513CF58392
:10179C00E58224091266F4127B05AD07AF56EF33D0
:1017AC0095E0FEEF7803C333CE33CED8F92436F56B
:1017BC008274003EF583EDF0AF55EF3395E0FEE516
:1017CC00522FF582E5513EF583E582240AF582E439
:1017DC003583F583E0FF127502AD07AF56EF3395F5
:1017EC00E0FEEF7803C333CE33CED8F92437F5823D
:1017FC0074003EF583EDF0D2688002C268AF5312DC
:02180C007B5C03
:01180E0022B7
:106FF000EF24FE601014601314601624037016D280
:1070000008D2248010D209D225800AD20ED226803E
:1070100004D20CD2277FF47E011279DD753D04E5A0
:107020003D70FC7F647E001279DDC224C225C22639
:0B703000C227C208C209C20EC20C2217
:045681008D51AC0794
:10568500C3EC648094815003025744EC6480948990
:105695004003025744E4F552AF51EF3395E0FEEF76
:1056A5007803C333CE33CED8F924E8F582741A3E95
:1056B500F583AF52EF3395E0FEE5822FF582E58362
:1056C5003EF583E0FD74182FF582741D3EF583EDDC
:1056D500F00552E552B408C0EC14FFAD511271A7A4
:1056E500D267AF51125AE3753D017F327E001279C0
:1056F500DDE53D70FCC267AF51125AE3E4F552E5B2
:1057050052FD3395E0FC74182DF582741D3CF5832C
:10571500E0FBAF51EF3395E0FEEF7803C333CE33B3
:10572500CED8F924E8F582741A3EF583E5822DF585
:0F57350082E5833CF583EBF00552E552B408C0E2
:015744002242
:046F06008D51AC07F6
:106F0A00D3EC64809480403CEC648094895035E4EE
:106F1A00FDECFF3395E0FEEF7803C333CE33CED8D2
:106F2A00F92428F58274003EF583EDFF3395E0FEDF
:106F3A00E5822FF582E5833EF583E4F00DBD08D1A5
:0B6F4A00D2688002C268AF51127B5C6D
:016F55002219
:04466A008C528D538E
:10466E00D3EF648094805003024772EF6480949578
:10467E004003024772EB648094875003024772EB4B
:10468E00648094E44003024772EF3395E0FEEF78C6
:10469E0005C333CE33CED8F92460F58274033EAF12
:1046AE0082F5568F57EB24FBF558D3940250030234
:1046BE004772E55875F00384E5F06003024772E532
:1046CE005875F00384F55AC39410400302477205DF
:1046DE0057E557AE567002055614F5828E83E55A8D
:1046EE00F074052553F553E43552F552E4F558E5CB
:1046FE0058C3955A506A855382855283E0F559B452
:10470E000A130557E557AE567002055614F5828EFC
:10471E0083E4F080120557E557AE56700205561425
:10472E00F5828E83E559F0855382855283A3E0FF8F
:10473E00855382855283A3A3E0FD1279768F5905A6
:10474E0057E557AE567002055614F5828E83E5591D
:10475E00F074032553F553E43552F5520558808F06
:0B476E00D2688002C268AF55127B5C6D
:01477900221D
:045745008F518D52A1
:10574900E551D3940050030257FCE55194154003E9
:105759000257FCD269AF52125A2F7D5F7F0512762C
:10576900B6AD51E4FF1276B67D527F041276B67F4C
:10577900F47E011279DD75F020E551A42460F582EB
:10578900E5F03403AF82F5558F56F583E0F55360A4
:105799004DD394004056E55394105050E55325E0FD
:1057A900F553755401E5532401FFE433FEC3E55471
:1057B9009FEE6480F87480985032E5562554F5823E
:1057C900E43555F583E0FFE5562554F582E4355572
:1057D900F583A3E0FD1276B60554055480C77D1BF9
:1057E9007F061276B67D5F7F051276B6C269AF5223
:0A57F900025A2FC268AF52127B5C07
:015803002282
:10775B008D51EFD3940A4006EFD3940F4003EF7093
:10776B000E90063FEFF0D268AF51127B5CD322C272
:08777B0068AF51127B5CC322D0
:107783008D51EFD3940A4006EFD3940F4003EF706B
:107793000E90063BEFF0D268AF51127B5CD322C24E
:0877A30068AF51127B5CC322A8
:1071ED008F55E555B40B067D5F7F078034E555B4AB
:1071FD000C067D5E7F068029E555B40D067D0A7F60
:10720D0002801EE555B40E067D327F028013E555D2
:10721D00B40F067D467F028008E55570077D0A7F15
:05722D00031276B622F9
:10765E008F51D269125A2F7D207F051276B67D2E5C
:10766E007F031276B67D527F041276B690063FE007
:0C767E00FF1271EDC269AF51125A2F22A9
:10768A008F51D269125A2F7D207F051276B67D213D
:10769A007F061276B67D527F041276B690063BE0DC
:0C76AA00FF1271EDC269AF51125A2F227D
:1078F0008D51D3EF64809480400EEF648094865065
:1079000007127446D2688002C268AF51127B5C22B3
:06736A008D51AB07AA06DD
:107370008B828A83A3A3A3E0FFEB2404F582E43A83
:107380001266F9D3EF648094804010EF648094A17A
:10739000500990063DEFF0D2688002C268AF5112EA
:0273A0007B5C14
:0173A20022C8
:067578008D51AB07AA06CD
:10757E008B828A83A3A3A3E0FFEB2404F582E43A73
:10758E001266F9EFC39421500990063CEFF0D268D1
:09759E008002C268AF51127B5C4F
:0175A70022C1
:065E25008E518F528B53D9
:105E2B00755406755540D3ED64809484407CED64C5
:105E3B008094A55075ED24FDF556D39404406BE585
:105E4B005620E06613F5570555E555AE547002051F
:105E5B005414F5828E83E557F074032552F552E402
:105E6B003551F551E4F556E556C3955750338552E8
:105E7B0082855183E0FFA3E0FD1279760555E55548
:105E8B00AC547002055414F5828C83EFF00552E587
:105E9B0052700205510552E55270020551055680AC
:105EAB00C6D268AF53127B5CD322C268AF53127B4E
:025EBB005CC3C6
:015EBD0022C2
:08477A008E518F528D538B54B8
:10478200C267D3E55364809484500302482FE553F3
:104792006480948D400302482F8F828E83A3A3E00E
:1047A200640A600302482F8F828E83A3A3A3E014BE
:1047B200B4080050769047C575F003A4C58325F070
:1047C200C583730247DD0247E70247F10247FB0256
:1047D200480502480F0248190248237555007556CC
:1047E20080D2678048755500755688D267803E75BD
:1047F2005500755690D2678034755500755698D21B
:1048020067802A7555007556A0D2678020755500BD
:104812007556A8D26780167555007556B0D2678056
:104822000C755500755678D2678002C267306750A2
:10483200E4FFEF7C002556FDEC35558D82F583E4CF
:10484200F00FBF08EDE55324FB855682855583F0B2
:104852007F01E5522404F582E43551F583E5822F88
:10486200F582E43583F583E0FEEF7C002556FDEC0E
:1048720035558D82F583EEF00FBF08D6D2688002DF
:07488200C268AF54127B5C19
:01488900220C
:04622D008E548F55A7
:106231000555E5557002055414F5828E83E0F55736
:106241006074C39408506F7F2C7E011279DDE4F5F0
:1062510056E556C39557505E855582855483E06057
:106261003624F5601414601714601A14601D14604C
:106271002024057028E4FD802D7D5F7F0780287D27
:106281005E7F0680227D0A7F02801C7D327F028034
:10629100167D467F0280107D0A7F03800A85558224
:1062A100855483E0FDE4FF1276B60555E55570028D
:0662B10005540556809B18
:0162B70022C4
:022D80008B5175
:102D8200C267EF640A6003022F5BED14B4080040CF
:102D920003022F59902DA475F003A4C58325F0C515
:102DA2008373022DBC022DF0022E24022E58022E15
:102DB2008C022EC0022EF3022F26D269AF51125A74
:102DC2002F7D577F021276B67D05E4FF1276B6E4B8
:102DD200FDFF1276B67D01E4FF1276B67D527F04C6
:102DE2001276B6755200755380D267022F5BD26994
:102DF200AF51125A2F7D577F021276B67D05E4FF3E
:102E02001276B6E4FDFF1276B67D02E4FF1276B6C4
:102E12007D527F041276B6755200755388D26702CE
:102E22002F5BD269AF51125A2F7D577F021276B6AD
:102E32007D05E4FF1276B6E4FDFF1276B67D03E46B
:102E4200FF1276B67D527F041276B6755200755324
:102E520090D267022F5BD269AF51125A2F7D577FF2
:102E6200021276B67D05E4FF1276B6E4FDFF127615
:102E7200B67D04E4FF1276B67D527F041276B675F3
:102E82005200755398D267022F5BD269AF51125A22
:102E92002F7D577F021276B67D05E4FF1276B6E4E7
:102EA200FDFF1276B67D05E4FF1276B67D527F04F1
:102EB2001276B67552007553A0D267022F5BD269A3
:102EC200AF51125A2F7D577F021276B67D05E4FF6D
:102ED2001276B6E4FDFF1276B67D06E4FF1276B6F0
:102EE2007D527F041276B67552007553A8D2678060
:102EF20068D269AF51125A2F7D577F021276B67D82
:102F020005E4FF1276B6E4FDFF1276B67D07E4FF14
:102F12001276B67D527F041276B67552007553B0A2
:102F2200D2678035D269AF51125A2F7D577F021274
:102F320076B67D05E4FF1276B6E4FDFF1276B67D25
:102F420008E4FF1276B67D527F041276B6755200FF
:102F5200755378D2678002C267306709AF53AE52A9
:102F620012622D8005AF51127988C269AF51125A8F
:012F72002F2F
:012F7300223B
:08315E008E518F528D538B54EA
:10316600C2678F828E83A3A3E0640A6003023215CE
:10317600124A9E8E568F57D3E557943BE5569400D8
:103186005003023210E5579408E5569407507BC366
:10319600E5536480948A5072855282855183A3A335
:1031A600A3E0F555B401069006000232BBE555B41E
:1031B60002069006020232BBE555B40306900604E9
:1031C6000232BBE555B404069006060232BBE5554D
:1031D600B405069006080232BBE555B4060690060D
:1031E6000A0232BBE555B4070690060C0232BBE56F
:1031F60055B4080690060E0232BBE555B409069092
:1032060006100232BBD267023337D26702333785E4
:103216005282855183A3A3E0640160030232C5ADE7
:1032260053AF52AE51124A9E8E568F57D3E55794DE
:103236003BE55694005003023337E5579408E556AC
:1032460094074003023337C3E5536480948A4003EE
:10325600023337855282855183A3A3A3E0F555B483
:103266000A05900612804EE555B4010590061480B5
:1032760044E555B40205900616803AE555B40305B3
:103286009006188030E555B4040590061A8026E5A8
:1032960055B4050590061C801CE555B40605900638
:1032A6001E8012E555B407059006208008E555B442
:1032B6000809900622E556F0A3806FD267807285D2
:1032C6005282855183A3A3E064027065AD53AF5269
:1032D600AE51126B687556008F57C3E5579463E578
:1032E600569400504CC3E5536480948850438552ED
:1032F60082855183A3A3A3E0F555B4010790063058
:10330600EFF0802DE555B40205900631801CE55599
:10331600B403059006328012E555B40405900633D1
:103326008008E555B40508900634E557F08002D2CA
:0F33360067306704C2688002D268AF54127B5CB4
:013345002265
:10267D008F518D528B53E551640A6003022729E572
:10268D0052C3940A40030228FFD269AF53125A2F46
:10269D007D277F081276B67D06E4FF1276B6E4FD3F
:1026AD00FF1276B6AD52E4FF1276B67D527F04125C
:1026BD0076B6E55214B4090040030228F89026D8E6
:1026CD0075F003A4C58325F0C583730226F3022696
:1026DD00F90226FF02270502270B022711022717F1
:1026ED0002271D02272390060002283990060202B8
:1026FD0028399006040228399006060228399006DA
:10270D000802283990060A02283990060C02283949
:10271D0090060E022839900610022839E551640101
:10272D006003022847E552D394004006E552940910
:10273D004009E552640A6003022844D269AF53127E
:10274D005A2F7D277F081276B67D06E4FF1276B6E6
:10275D00E552B40A147D0AE4FF1276B67D527F0469
:10276D001276B6900612022839E552B401147D0B8B
:10277D00E4FF1276B67D527F041276B690061402EF
:10278D002839E552B402147D0CE4FF1276B67D5261
:10279D007F041276B6900616022839E552B403135B
:1027AD007D0DE4FF1276B67D527F041276B690064B
:1027BD00188079E552B404137D0EE4FF1276B67DD0
:1027CD00527F041276B690061A8061E552B4051355
:1027DD007D0FE4FF1276B67D527F041276B6900619
:1027ED001C8049E552B406137D10E4FF1276B67DC8
:1027FD00527F041276B690061E8031E552B407134F
:10280D007D11E4FF1276B67D527F041276B69006E6
:10281D00208019E552640860030229067D12FF121B
:10282D0076B67D527F041276B6900622E0FEA3E0C6
:10283D00FF1275470229060228FFE5516402600365
:10284D00022906E552D3940050030228FFE5529465
:10285D000740030228FFD269AF53125A2F7D277FFD
:10286D00081276B67D06E4FF1276B67D14E4FF12EB
:10287D0076B6E55224FE602014603014604014607A
:10288D0050240470667D01E4FF1276B67D527F04FC
:10289D001276B6900630804A7D02E4FF1276B67D40
:1028AD00527F041276B690063180377D03E4FF1215
:1028BD0076B67D527F041276B690063280247D0462
:1028CD00E4FF1276B67D527F041276B69006338001
:1028DD00117D05E4FF1276B67D527F041276B69017
:1028ED000634E0FF7E001275A8800EAF5312798872
:1028FD008007C268AF53127B5CC269AF53125A2F67
:01290D0022A7
:064A9E008E588F59A90596
:104AA4007D057C00E5592DF582E5583CF583E0C38E
:104AB400940A400CE5592DF582E5583CF583E4F061
:104AC4000DBD00010CED640A4C70D9B90610E5590E
:104AD4002405F582E43558F583E0FF7E0022E9647D
:104AE400077019E5592405F582E43558F583E07516
:104AF400F00AA4ACF0FDE55924068032E96408709C
:104B04003DE5592405F582E43558F583E075F064F4
:104B1400A4ACF0FDE5592406F582E43558F583E0AC
:104B240075F00AA42DFDE5F03CFCE5592407F58257
:104B3400E43558F583E02DFDE43CAF05FE22E9643D
:104B440009705AE5592405F582E43558F583E0FFE8
:104B54007E007C037DE81258E2AC06AD07E55924DB
:104B640006F582E43558F583E075F064A42DFDE57F
:104B7400F03CFCE5592407F582E43558F583E075EB
:104B8400F00AA42DFDE5F03CFCE5592408F582E487
:104B94003558F583E02DFDE43CFEAF0522E4FEFF2D
:014BA40022EE
:066B68008E588F59A905AB
:106B6E007F057E00E5592FF582E5583EF583E0C39B
:106B7E00940A400CE5592FF582E5583EF583E4F072
:106B8E000FBF00010EEF64084E70D9E96407702044
:106B9E00E5592405F582E43558F583E075F00AA42D
:106BAE00FFE5592406F582E43558F583E02FFF22E0
:026BBE007F0056
:016BC00022B2
:104BA5008F56E556D3945940147D5AE4FF1276B6D4
:104BB500E55624A6FD7003024CA6024CA1E556D38A
:104BC500944F401AE556945A50147D50E4FF1276DE
:104BD500B6E55624B0FD7003024CA6024CA1E5567D
:104BE500D39445401AE556945050147D46E4FF127F
:104BF50076B6E55624BAFD7003024CA6024CA1E533
:104C050056D3943B4019E556944650137D3CE4FF3A
:104C15001276B6E55624C4FD7003024CA6807DE5E8
:104C250056D394314016E556943C50107D32E4FF3E
:104C35001276B6E55624CEFD60678060E556D394BE
:104C4500274016E556943250107D28E4FF1276B6BB
:104C5500E55624D8FD604A8043E556D3941D401699
:104C6500E556942850107D1EE4FF1276B6E55624CD
:104C7500E2FD602D8026E556D394134016E5569443
:104C85001E50107D14E4FF1276B6E55624ECFD6047
:104C9500108009E556C394145007AD56E4FF12760B
:024CA500B62235
:1075A8008E548F557C007D0A1258F4AD07E4FF1203
:1075B80076B67D5B7F061276B6AE54AF557C007DFD
:1075C8000A1258F4E4FF1276B67D4A7F070276B6AF
:047547008E548F557A
:10754B007C007D3C1258F4124BA57D057F0612760C
:10755B00B6AE54AF557C007D3C1258F4ED4C600C2C
:0C756B00AF05124BA57D4A7F071276B6D3
:0175770022F1
:027085008D512B
:10708700D3EF648094804038EF648094955031EF5B
:107097003395E0FEEF7805C333CE33CED8F92460BD
:1070A700F58274033EAF82FEE4FD0FEFAA0670017E
:1070B7000E14F5828A83E4F00DBD20EED2688002BB
:0770C700C268AF51127B5CAF
:0170CE00229F
:1072F1008F51900640E0D394024015D267125AE3B1
:10730100753D037F327E001279DDE53D70FC80150D
:10731100D267AF51125AE37D1B7F061276B67D0C00
:0D7321007F031276B6C267AF51125AE32205
:107B2A007E10900640E4F0A3DEFC7E10D268127B41
:017B3A005CEE
:017B3B002227
:107869008F5CD269125A2F7D607F021276B67D3203
:107879007F061276B67D1E7F051276B6C269AF5CA9
:04788900125A2F223E
:107988008F5CD269125A2F7D607F021276B67D30E5
:0D7998007F031276B6C269AF5C125A2F222F
:0E7B5C008F5B306803027869AF5B1279882274
:1066B6002432F58274003EF583EDF0AF55EF339545
:1066C600E0FEE5522FF582E5513EF583E58224048E
:1066D600F582E43583F583E0FFE555FD3395E0FC6F
:1066E600E5522DF582E5513CF583E5822405F582D8
:0766F600E43583F583E0FDAC
:1066FD00EFD394004015EF940B5010EFC3940A5054
:10670D0008EF75F00AA4FE8002E4FEEDD39400407C
:10671D000EED940B5009EDC3940A5003ED2EFEAF10
:01672D000665
:01672E002248
:03000000027B4D33
:0F7B4D00758E0078FEE4F6D8FD75816C02517AD2
:107A7400D292C0F075F008C29100A29233D291D58F
:067A8400F0F5D0F0FF2236
:107A8A00EFC0F075F00833C291929333D291D5F0DA
:067A9A00F6D0F0C29122BB
:1076B600EFFEEDFF1280008E2F8F30125CE2755FB9
:1076C60064AF5F155FEFD39400400EE4F55EE55EB0
:0976D600C3943A50EC055E80F506
:0176DF002288
:105CE200D2A885A86175A881C244853082852F8398
:105CF200E493F560C4540FF5604360F0856080C2A0
:105D020084D28500C2870000D287007580FF75802B
:105D1200FEC284C28500C28700000000D2870075DF
:105D220080FFD24475623E756380E4F56030941D55
:105D32000560E560B464F6123346E56315637002EC
:105D42001562D3E5639400E562940050DD75623E0E
:105D5200756380E4F56020941D0560E560B464F627
:105D6200123346E563156370021562D3E56394004E
:105D7200E562940050DD8561A8C2A87F147E0012FE
:025D820079DDC9
:015D840022FC
:1076E0007580FDC284C28500C28700000000D28779
:1076F000007580FF7F147E001279DD7F997E09126C
:0A77000080008E2F8F30125CE22211
:1058C000C2D530F707B2D563F0FF05F030E70CB270
:1058D000D5F4048463F0FF05F080018430D502F430
:0258E0000422A0
:1058E200EF8DF0A4A8F0CF8CF0A428CE8DF0A42EDA
:0258F200FE2294
:1058F400BC000BBE0029EF8DF084FFADF022E4CC98
:10590400F875F008EF2FFFEE33FEEC33FCEE9DEC60
:10591400984005FCEE9DFE0FD5F0E9E4CEFD22EDA6
:10592400F8F5F0EE8420D21CFEADF075F008EF2FF0
:10593400FFED33FD4007985006D5F0F222C398FDE1
:055944000FD5F0EA227E
:10594900EB9FF5F0EA9E42F0E99D42F0E89C45F0B4
:01595900222B
:10595A007401FF3395E0FEFDFC080808E6CF2FF638
:10596A0018E6CE3EF618E6CD3DF618E6CC3CF62211
:107B3C00EFC39461400AEF947B5005EF24E0FF22E1
:017B4C002216
:00000001FF
